:040000006F00204429
:100004000000000000000000480200004A02000056
:100014000000000040040000000000000000000098
:100024004004000040040000000000000000000044
:10003400701A0000000000004004000000000000EE
:10004400400400004004000040040000400400009C
:10005400400400004004000040040000400400008C
:100064003815000040040000400400004004000073
:10007400400400004004000040040000400400006C
:10008400400400004004000040040000400400005C
:10009400400400004004000040040000400400004C
:1000A400400400007E1A00004004000040040000E8
:1000B400461A0000961900004004000040040000A5
:1000C400400400004004000040040000400400001C
:1000D4004004000040040000400400008A180000AE
:1000E40040040000400400004004000040040000FC
:1000F40040040000D0180000400400004004000048
:1001040040040000400400004004000040040000DB
:100114004004000000000000000000000000000097
:1001240000000000000000000000000000000000CB
:0C013400000000000000000000000000BF
:10014000397101436EC619A0397141536AC866CA34
:1001500062CC5ECE19A0397101535AD056D252D416
:100160004ED64AD826DA22DC06DE3301614082828E
:1001700041114AC026C222C406C68282B24D410144
:10018000024D924C224CB24B4101024B924A224A00
:10019000B2494101024992442244B2404101828065
:1001A0003D432A876373C3029377F700BDEFADE544
:1001B000937606FF3D8ABA960CC34CC30CC74CC756
:1001C0004107E36BD7FE11E28280B306C3408A0683
:1001D0009702000096966780A6002307B700A30643
:1001E000B7002306B700A305B7002305B700A30493
:1001F000B7002304B700A303B7002303B700A3028B
:10020000B7002302B700A301B7002301B700A30082
:10021000B7002300B700828093F5F50F9396850011
:10022000D58D93960501D58D61B7939627009702DA
:10023000000096968682E78086FA9680C1171D8F09
:100240003E96E374C3F8A5B701A001A0EFF25FF2F8
:100250000545EF00D0289922EF101018716513059D
:100260000520EF10D01CB707002083A507163775AF
:1002700000001305C537EF5070650925AA8537754D
:1002800000001305C538EF507064EF30204AEF309E
:10029000A041014501B7EFF2BFED371402401C4009
:1002A0003707FF08411193E717001CC05C40F98F26
:1002B0005CC01C403707F7FE6D17F98F1CC01C404F
:1002C0003707FCFF7D17F98F1CC05C40370701FF23
:1002D0007D17F98F5CC0B7079F001CC4EF00300783
:1002E00002C402C6B7270240054798C31C404167B5
:1002F000B7160240D98F1CC03706020005679C4222
:10030000F18F3EC6A24785073EC4B24781E7A247A8
:10031000E397E7FEB71702409C431397E700635744
:10032000070685473EC6324785476313F706B7176A
:100330000240D843B706C1FFFD16D8C3D843D8C37F
:10034000D84313670740D8C3D843758FD8C3D84361
:10035000B7061100558FD8C39843B7060001558FD3
:1003600098C3984393166700E3DD06FED843B7169B
:100370000240719BD8C3D84313672700D8C32147D5
:10038000DC42B18BE39EE7FE410129B502C661BFA5
:10039000372702401C43F19B1CC3FDB7B716024030
:1003A000DC42370700201146B18B13070716638F15
:1003B000C70221466381C70495EB9C42918B9DC780
:1003C000B7470F00938707241CC3B7170240DC43CD
:1003D000918393F6F700B707002093870700B6973D
:1003E00094231C43B3D7D7001CC38280B7177A006D
:1003F00093870720D1BFDC42D4424166C983BD8BBD
:10040000F18E890745466393C700C94781EEB74619
:10041000024083A60680C18A89CEB7167A009386E9
:10042000062021A8B7160240D4421396E600E356F0
:1004300006FEB7163D0093860690B387D70269B7CC
:1004400001A0970100209381E15117510020130171
:1004500061BB178500001305A590970500209385C3
:1004600065BA1386018263FAC5008322050023A0C2
:10047000550011059105E3EAC5FE138501829385B8
:10048000C1B66377B500232005001105E36DB5FE05
:10049000FD42739002BC8D427390428093028008AB
:1004A0007390023097020000938202B693E232000A
:1004B00073905230EFF03FDE97020000938242D9F2
:1004C0007390123473002030B727014093870740A0
:1004D000631FF500EFF2DFC9854513050020EF002B
:1004E0001018814513050020EF00701765B1828058
:1004F0005C413707F1E01307F7EF944D7D8F9C4186
:10050000D58FD44DD58FD441A206D58FD98F5CC15C
:100510001C4537F7F1FF1307D77FD4457D8F9C49E2
:10052000D58F94458606D58FD98F1CC55C55370766
:1005300010FF7D177D8FDC29FD1793F7F70FD2078A
:10054000D98F5CD582801C4589C593E717001CC5EF
:100550008280F99BEDBF1C4593E787001CC5828014
:1005600008450D81058982801C4593E747001CC51D
:10057000828008450981058982801C4591C537071D
:100580005000D98F1CC582803707B0FF7D17F98FC7
:10059000D5BFA54763F7B7048D47138765FF3307BA
:1005A000F7020328C5009D47B397E70093C7F7FFFD
:1005B000B3F70701B396E600DD8E54C5994763E3B0
:1005C000C70495477D163306F6025859FD47B39781
:1005D000C70093C7F7FFF98F3396C5005D8E50D9DA
:1005E00082800D473387E502032805019D47B397B5
:1005F000E70093C7F7FFB3F70701B396E600DD8E78
:1006000014C96DBFB14763E2C7029547651633064B
:10061000F6021859FD47B397C70093C7F7FFF98F44
:100620003396C5005D8E10D9828095474D163306EE
:10063000F6025855FD47B397C70093C7F7FFF98FE8
:10064000B395C500DD8D4CD582806845420541815A
:10065000828008416D8D3335A00082805C4191C558
:1006600037070004D98F5CC18280370700FC7D17F3
:10067000F98FD5BF3C4989C593E707083CC98280FB
:1006800093F7F7F7E5BF3C4989C593E707043CC9F1
:10069000828093F7F7FBE5BF3C4993F7F7FD3CC930
:1006A0003C49DD8D2CC98280EFF29FACB7066745CF
:1006B000B7270240938636123797EFCDD4C313077E
:1006C000B79AD8C3D4D3011198C7D45B1387470313
:1006D00013962600E34B06FED45737250140130539
:1006E000054093E60620D4D7DC5BB7060020D58F03
:1006F0001CC31C431C4537070E00D98F1CC51C4565
:1007000093E717001CC53C4993E707043CC91C4507
:1007100093E787001CC52A842285993575FD372506
:100720000140832785401305054093E747001CC51A
:100730002A8422853D3D75FD372501400546C94582
:10074000814613050540B1352546230401003727AE
:100750000140B70550001C84637FF60423040100A8
:10076000A54621461C8463FFF606231501002304D9
:10077000010095461C8463F1F60E38853C85994648
:100780000D46B3F7D7020565130505803357D70229
:10079000B3D7C702BA97C207C1837C85B727014088
:1007A00003A78740799B23A4E7403C8505611D8D05
:1007B00042054185C5B283278740CD8F2324F7406A
:1007C00083270740898BEDDF1C848326C7440810EC
:1007D0008607AA972396D7FE1C84850793F7F70F01
:1007E0005C8495BFA30401009C846378F6001C849C
:1007F000850793F7F70F5C84B5B798849C840C1039
:100800000607850786072E97AE970357C7FE83D73F
:10081000C7FE63FDE7029C848607AE9783D7C7FEB9
:100820007C859C84988485078607AE9783D5C7FE10
:10083000931717001810BA972396B7FE9C84388533
:100840000C1085078607AE972396E7FE9C848507E4
:1008500093F7F70FDC8449BF1C8410103885890793
:100860008607B29783D7C7FEBA97C207C1837C8534
:100870001C84850793F7F70F5C84EDBD03A54182C7
:1008800082805841032805004C45370601409307F4
:1008900006403E979346F8FFB1C583250640F58D87
:1008A0002320B640D043F18ED4C31443B3E60601EF
:1008B00014C3184190479346F7FF758E90C7D047F1
:1008C000F18ED4C7144541466399C6009447D98E2A
:1008D00094C7D447558FD8C78280B6979443558F15
:1008E00098C382801C43F58F1CC38280B7070140E8
:1008F0001387074083A70740584B698F09C77D8D31
:100900003335A000828001458280B707014023AAC9
:10091000A74082809C4513F7070113F8F70001C731
:10092000D8413368E8008E2113F7F50F39C3184119
:100930008146854E3D4F930F800293028004214EE5
:100940003396DE00B3F8C5006311160393982600B2
:1009500033131F011343F3FF3377E300B318180178
:1009600033E7E800639FF70550C98506E39AC6FDA3
:1009700018C11307F00F6375B70454412146854E23
:100980003D4F930F800293028004414EB398CE00F6
:1009900033F715016392E80213172600011733138A
:1009A000EF001343F3FFB376D3003317E800D98E7B
:1009B000639DF701232A15010506E319C6FD54C1FD
:1009C0008280E39457FA10C94DB7E39757FE232866
:1009D0001501DDB708456D8D3335A000828048458F
:1009E0006D8D3335A00082800CC9828019C20CC97C
:1009F00082804CC98280370700C0B377E5006395D9
:100A0000E708370701405C439356B501584F9D8A6C
:100A10009DE6F99BB70600FFFD16758F89C99316F1
:100A20000501C182D58FB706FF01758D498FB706C5
:100A30000007D58FB7060140DCC2D8CE82800546BC
:100A40006396C600F59BB70680FFF9B70946639623
:100A5000C600ED9BB706E8FFC1B70D466396C6001A
:100A6000DD9BB706FCFF4DBF11466397C60093F7A9
:100A7000F7F3B706C0FF4DB71546E391C6FA93F7F3
:100A8000F7CFB706E0FF49BF370700406391E702A1
:100A9000B7070140D84F4205B367A70089E5134562
:100AA000F5FFB377E500370701405CCF8280A9E30B
:100AB00037080140B7073000032648001317050127
:100AC000B376F50041836396F602B70600F9FD168A
:100AD000B377D60003264800F18E2322D80091C5B3
:100AE000558112053315A700C98F370701405CC334
:100AF00082809317B50063D007029357050193F6E0
:100B0000F7008D47B397D70093C7F7FFF18FB7066C
:100B10000007D58FE9B7935755019207B317F70030
:100B2000E5B713F7C50F93F73500B7050140BA9540
:100B300094458A073D473317F7001347F7FF758F32
:100B400098C598453315F500598D88C58280EFF218
:100B50002FE237F4FF1F032744723706003E41118E
:100B6000931797019346F7FFF18F060737063E006C
:100B7000718FD98F3706000113979600718FD98F27
:100B8000BD824167F98ED58F02C202C402C623A47A
:100B9000F1820357847285452390E1820327047212
:100BA0001305D00323A6E1820327447023A2E18228
:100BB0008D2C8327447037073A101307077093F77B
:100BC000F7F06380E7106361F7023707321013070D
:100BD00007706380E70637073710130707706387CE
:100BE000E70841016FF00FDB37073B101307077071
:100BF000638BE70A37073D1013070770E393E7FE9F
:100C000085452165CD3BB7140140E177130480048D
:100C10004C00138504807C8222C6ED39856793875A
:100C2000C7334C00138504C07C8222C6E531F977B6
:100C30000DA085452165C133B7140140930700E03D
:100C4000130480044C00138504C07C8222C6D93171
:100C500089674C00371501407C8222C665398D4773
:100C60007C8222C64C001385044025A8B71401409D
:100C7000E17793870770130480044C001385048088
:100C80007C8222C641399307D0E34C00138504C00F
:100C90007C8222C64131F9777C8222C64C0037150E
:100CA00001408D393DBFB7140140E1771304800442
:100CB0004C00138504807C8222C6A939930740200A
:100CC0008DB7B7140140E177130480044C001385FD
:100CD00004807C8222C63D398967F51799B723A81D
:100CE000A182828003A70183854714216310F70244
:100CF0001C31639CE7023C21960793E707F837E72E
:100D000000E093F7F70F36972300F740054793D796
:100D100056003317D700544189CE938707048A07BA
:100D2000B7E600E0B69798C38280EDF33C219607C2
:100D3000F9B793870706E5B7B7160240DC42374795
:100D4000FF7F7D17F98F5D8DC8C282803717024003
:100D50005C439146B18B638CD706A146638ED70660
:100D6000BDE71C43918BA5C7B7470F0093870724A6
:100D70001CC1371602405C423707002013070701E9
:100D80009183BD8BBA9794231C41B3D7D7005CC124
:100D90005442A1829D8ABA969422B3D6D70014C534
:100DA0005442AD829D8A36971423B3D6D70054C5DA
:100DB0005842634C07005C42B98313F737009387AE
:100DC0004180BA979C23B3D7F6021CC98280B7171B
:100DD0007A009387072069BF5C435843C166C98383
:100DE000BD8B758F8907C5466393D700C94701EF4F
:100DF0003747024003270780418B09CF37177A0016
:100E00001307072021A83717024058439316E7001D
:100E1000E3D606FE37173D0013070790B387E702B6
:100E200081BF99C5371702401C4F5D8D08CF828066
:100E3000B7170240984F1345F5FF798D88CF828010
:100E400099C5371702405C4F5D8D48CF8280B71738
:100E50000240D84F1345F5FF798DC8CF828099C5E0
:100E6000371702405C475D8D48C78280B717024044
:100E7000D8471345F5FF798DC8C782801A218D6741
:100E800093870704B6217D8F9E21D58FD621D58FDC
:100E9000F621D58F9625D58FB625D58FD625D58F1A
:100EA000F625D58FD98F1EA19E291EA982801E21CD
:100EB00089C593E707041EA18280C207C18393F707
:100EC000F7FBC207C183C5BF4EA582804A25828039
:100ED0000A256D8D3335A00082801E2137370140F1
:100EE000130707C0C207C1836300E502370700404C
:100EF000630CE500130707406308E500371700405F
:100F0000130707806316E500FA2193F7F7F8D98FE6
:100F10009A2593F7F7CFC207C183D98F37170040BF
:100F20001EA1130707809C416310E5025CD5DE21FA
:100F30001EB5B7370140938707C06314F500BC2581
:100F40001EB985475EA98280C207C1835EB5C5B759
:100F50001A31FD77FD17F98F1EB10358050256218E
:100F60005E2D6577D2211307F7CF7D8FF9772206A3
:100F7000FD17518FB3F70701F22103D8A500C20670
:100F80004207336606013206D18F37360140C20769
:100F9000130606C0C1824183C183631AC5007176FE
:100FA0007D16F18EF2251A06D18EC206C18256A197
:100FB000B71600405AAD9386068098416315D50058
:100FC00038C11EB1828042074183DDBF1E2189C521
:100FD00093E717001EA18280C207C183F99BC20755
:100FE000C183CDBF8357450491C52167D98F231293
:100FF000F5048280C607C583DDBF5E2501C6DD8D91
:101000004EA5828093C5F5FFFD8DDDBF1E2189C5EC
:1010100093E707081EA18280C207C18393F7F7F701
:10102000C207C183C5BF5A2DFD779387F77FF98F1C
:10103000A205CD8FC207C1835EAD8280B717004085
:10104000938707806314F5002CC18280C205C1819B
:10105000E5BFB7170040938707806314F500485138
:1010600082804A314205418182801E294A25ED8FC6
:101070004205418189C76D8D3335A00082800145CD
:10108000828093C5F5FFC205C1810EA98280EFF26F
:101090002F8E1629F577FD17F58FF621DA25797150
:1010A000D58F1EA95625FD779387379FF58FD621BB
:1010B0002A842EC6D58F9625D58FB625D58F5EA5C9
:1010C0005E29C207C18393F7F7CFD98F5EA968085D
:1010D000B539B747014093870780B245631AF404D6
:1010E000A25756246547B387E702C206C1869841D6
:1010F00063D20604060752244206B3D7E702130759
:1011000040064186B3D6E702B3F7E702920663557D
:1011100006028E0793872703B3D7E70213F77700FA
:10112000B367D700C207C1831EA445616FF08F86E5
:10113000925745BF0A07C1B7920793872703B3D7D2
:10114000E702BD8BD58FF9BF91C55E250967D98FA1
:101150005EA582805A25F977FD17F98FD5BF13F761
:10116000F50F85471583B395B7006319F70093070B
:10117000C500984301CED98D8CC3828089469307E0
:101180004501E318D7FE93070501E5B793C5F5FFC1
:10119000F98DDDB793F5F51F4EA182804A211375B5
:1011A000F51F82800A216D8D3335A000828013F7F0
:1011B000F50F85461583B397B6006311D7025A25FC
:1011C000F98F1A2101454207418381CB0545A18151
:1011D000B315B5006D8F3335E00082808946631406
:1011E000D7001A29F1BF5A29E1BFEFE27FF87971E0
:1011F0001306000281450808EFE09FFA8545114576
:1012000002C202C402C631398545130500201139D6
:1012100001451D36371501409307E00F4C001305BB
:101220000580372401407C8202C6EFF0AFEE130543
:101230000440EFF06FA913050440EFF0EFC6AA8554
:10124000239AA182377500001305C539EF40106855
:10125000B7070E003ECE0C08854713050440230255
:10126000F10202C802CA02CC02D0EFF06FA8854595
:1012700013050440EFF02FAD854513050440EFF052
:101280008FC0814513050440EFF04FBD13050440A6
:10129000EFF06FAC930404402685EFF06FAC6DFD6A
:1012A0001305044037240140EFF00FAC93040440D1
:1012B0002685EFF00FAC6DFD37050080B53C1305BA
:1012C00004408545EFF00FBB930500021305044071
:1012D000EFF08FBC45616FE0FFEBEFE27FE90111BA
:1012E000854521453D3E85451165993E37140140B0
:1012F00085678D447C808A85C147130504C03EC440
:1013000026C2EFF02FE1130504C08565EFF0CFEDA5
:10131000896761498A85130504C07C804AC426C256
:10132000EFF04FDF91677C808A859147130504C0F9
:101330003EC4EFF02FDEE1778A85130504C07C8080
:101340004AC426C2EFF00FDDB70704013EC6B70757
:1013500002003EC8B70700028507374400403ECA76
:10136000A1473ECC6C009D4713050480FC863936AE
:10137000854513050480253E05616FE0BFE1EFE27E
:101380009FDDB74400402A891304900C93890480A0
:1013900089454E85353E0DC5CA8513850480B74401
:1013A00000401D361304900C1389048085454A853E
:1013B000053611CD13850480113E1375F50F31A04C
:1013C0007D141374F40F69F401456FE01FDC7D1484
:1013D0001374F40F61FCCDBFEFE29FD92A89371552
:1013E00001402E84130505C08565B2840146EFF0E7
:1013F000EFDF0D456937135504011375F50F4137BC
:10140000135584001375F50F9D3F1375F40F853F39
:10141000014493170401C18363EC97003715014021
:1014200005468565130505C0EFF04FDC6FE09FD6DC
:101430001305F00FA937B307890088A30504D1BFAE
:10144000EFE21FD3411185451145E13A93070010A2
:101450007C8237150140C1473EC64C008D471305BD
:1014600005803EC4EFF00FCB41016FE0BFD2EFE249
:101470003FD0411185454145EFF0BF9A856793877D
:1014800007807C8237150140C1473EC64C008D471E
:10149000130505803EC4EFF0EFC741016FE09FCF19
:1014A000EFE21FCD411185452145EFF09F9793074E
:1014B0000010371401407C82C1473EC64C008D4766
:1014C000130504C03EC4EFF0EFC4054693050010B9
:1014D000130504C0EFF08FD141016FE0BFCBEFE205
:1014E0003FC9797185452545EFF0BF939147371581
:1014F0000140FC824C0893078004130505C03ECED2
:10150000EFF04FC189450545EFF0AFE19147054444
:101510003ED00810B1473ED422D602D2EFF06FB6CB
:10152000930780117C86680089475C8722C8EFF0AA
:101530006FFB45616FE01FC64111114522C626C4ED
:101540004AC2EFF0AFBA85476318F5043719014076
:10155000AA8401469145130509C0EFF02FC983C73E
:10156000018895E705469145130509C0EFF00FC8BE
:10157000238091883715014001469305001013051B
:1015800005C0EFF0AFC689472380F18819A0E38337
:1015900097FE1145EFF06FB73244A2441249410162
:1015A00073002030EFE2DFBC411185452145EFF0AB
:1015B0005F87A147371401407C82C1473EC64C007B
:1015C0008D47130504C03EC4EFF0CFB40146A145DA
:1015D000130504C0EFF08FC141016FE0BFBBEFE224
:1015E0003FB9411185452145EFF0BF838545114540
:1015F000EFF01F8593070020371401407C82E147FC
:101600003EC64C008D47130504C03EC4EFF08FB0BA
:10161000930700084C00130504C07C82EFF08FAFE5
:1016200041016FE03FB7EFE2BFB401114D3F371406
:1016300000409307F01D8A85130504803EC002C256
:101640002314010023050100EFF03F8913050480F6
:101650008545EFF0BF9BC167938707066C001305B4
:1016600004803EC8231B010002C6EFF07F8E1305E5
:101670000480A145EFF03F9B130504808545EFF002
:10168000FF94854513050480EFF0DF9505616FE059
:101690007FB0EFE2FFADB7770000044103A9473BFD
:1016A0002A842685CA85EF30D05F6358050223203F
:1016B0002401B777000083A5C73B0840EF303067AF
:1016C000EF40C04E9315050137150040C181130549
:1016D0000580EFF0BF966FE0FFAB2685EF40A06B73
:1016E000B777000003A6073C83A6473CEF20901481
:1016F000E351A0FCB777000083A7873B1CC055BF10
:10170000EFE21FA7797137140140C1472A89FC8293
:101710008D44C1474C08130504C03ECE26CCEFF0E3
:101720006F9F0146130504C0C145EFF02FAC8545FE
:101730002145EFF00FEF854537050800EFF04FF03A
:101740008547FC824C08E147130504C026CC3ECEF9
:10175000EFF04F9C894491474C08130504C0E48284
:10176000375400403ECEEFF0EF9A0C10B7070C0054
:10177000130504C04AD03ED402D223160102EFF072
:101780001F919307D0137C86680085473EC8448725
:10179000EFF04FD50546130504C093055052EFF006
:1017A0001F9C8545130504C0EFF01F9A45616FE04B
:1017B0007F9EEFE2FF9B797137140140930700028F
:1017C0002A89FC828D44C1474C08130504C03ECED3
:1017D00026CCEFF02F940146130504C093050002B8
:1017E000EFF0CFA085452145EFF0AFE38545370504
:1017F0000400EFF0EFE493070040FC824C08E1475F
:10180000130504C026CC3ECEEFF0CF9085679387BA
:101810000780FC824C089147130504C03ECE375424
:101820000040EFF02F8F0C10B7070C001305048059
:101830004AD03ED402D223160102EFF05F8593070F
:1018400070137C8685475C87680085473EC8EFF04B
:101850006FC905461305048093055052EFF03F9081
:10186000854513050480EFF03F8E45616FE09F9240
:10187000EFE21F902A84EFF0FF9193050008228584
:10188000EFF05F927DD96FE0FF90411122C637548F
:1018900000409305505213050480EFF05F910DC591
:1018A00013050480EFF09F8F9375F50F238CB182A1
:1018B00003A581881C4D104954498507B3E7C70229
:1018C0006384D7003105452C324441017300203038
:1018D000411122C63754004093055052130504C0ED
:1018E000EFF0FF8C0DC5130504C0EFF03F8B93752F
:1018F000F50F238EB18203A5C1881C4D10495449B0
:101900008507B3E7C7026384D7003105AD243244AD
:10191000410173002030EFE2BF850111AA842E84BB
:1019200009458545EFF0CFD1E084370400404C08ED
:101930001305044026CA231E0100231D0100EFF0F9
:10194000CFD90546854513050440EFF00FEB93070B
:10195000D0027C8685475C87680085473EC8EFF0EB
:101960006FB805616FE01F83EFE29F80B70700202B
:1019700083A50716896793870771B3D5F502A94731
:101980003305F502FD15C205C1817D154205418172
:1019900059376FE03F80411122C63704004085452A
:1019A00013050440EFF06FEC01C9854513050440B1
:1019B000EFF02FEDEF00B0373244410173002030DB
:1019C000EFE20FFB01112E84AA8485450545EFF057
:1019D0002FC74C083705004026CAE084231E0100AB
:1019E000231D0100EFF06FCF054685453705004008
:1019F000EFF0AFE09307C0027C868D475C876800FC
:101A000085473EC8EFF00FAE854537050040EFF043
:101A1000EFDB05616FE00FF8EFE28FF5B70700200D
:101A200083A50716896793870771B3D5F502A94780
:101A30003305F502FD15C205C1817D1542054181C1
:101A400041376FE02FF5854537050040EFF0EFE1B6
:101A500011CD854537050040EFF0AFE2CD2083C6BC
:101A6000018805476394E6002380018873002030D5
:101A7000B7F700E023A20700D920730020304111FE
:101A800022C6373401408545130504C0EFF0EFDD71
:101A900001CD130504C08545EFF0AFDE37750000BA
:101AA0001305853CEF40C073324441017300203080
:101AB0001DC9B296C206C18252A136A10CC509EE5B
:101AC00085471CA183A6018493870184368701EB97
:101AD00054C588C30145828023000500E5B763062D
:101AE000A7005847EDB77D558280054582800DC51A
:101AF00083A701841387018499E305458280D44735
:101B00006396A6005845D8C7014582806394A70014
:101B100014C3DDBFB687CDB77D558280EFE24FE5B8
:101B200003A4018475DC1C2093F7F70F99C75E208E
:101B300099C3230004001C4482974044E5B783A75F
:101B40000184054691E38280D62381CEBA237D1796
:101B500042074183BAA3BA234207418319E390A302
:101B6000B6A3DC47C5B7232605000CC150C123240A
:101B70000500054582805C45544118458507B3E75B
:101B8000D702638EE70058451C41BA978CA35C4589
:101B900058418507B3E7E7025CC505458280795562
:101BA000828018455C45630FF70018451C41BA97C1
:101BB0009C239CA11C4558418507B3E7E7021CC53F
:101BC00005458280014582805C4518454841998FD2
:101BD000AA9733E5A7028280B707002083A70716DC
:101BE0000967130707F4B3D7E702C207C18323933A
:101BF000F1842392F1848280B7F700E0D8438146D4
:101C0000799BD8C303D741843306A70290CBD4CBAA
:101C100098431367070198C398431367170298C343
:101C2000D843058B75DF9843799B98C38280EFE298
:101C30002FD42A841165011185451105EFF06F9E9F
:101C4000930700207C82371501408D473EC44C002D
:101C5000E147130505803EC6EFE0DFCB22C83744DD
:101C60000140B70708000C08130504803ECC02CAE7
:101C7000231E0100EFF0AFC1854513050480EFF08E
:101C8000AFCC05616FE00FD1EFE2EFCCB74401407C
:101C9000AE893289014493840480634524014A85D6
:101CA0006FE0AFCE930500042685EFF0AFCF7DD96E
:101CB000B38789008385070026850504C205C18195
:101CC000EFF04FCDD9BF138781801C439386C1B6F7
:101CD0003E95636BD500B75600209386068063E57A
:101CE000A60008C33E858280FD57EDBFEFE24FC8D6
:101CF00037240140AA859546054613050440EFE0C8
:101D00005F89854513050440EFE03F879304044055
:101D100089452685EFE0FF9365DD13050440EFE07C
:101D2000DF926FE02FC70397418381472A97634F64
:101D3000070009CD05669306F6FFB6876358C7000E
:101D4000AA876305D50093170701C1833E8582806A
:101D5000EFE20FC20545593F42054185E937EF30B3
:101D6000B076B777000083A5873DEF300040EF40A5
:101D70008002B777000003A6073E83A6473EEF2008
:101D8000A041B777000003A6873E83A6C73EEF2099
:101D9000A0402A86AE86EF10F036EF40800A6FE052
:101DA0006FBFEFE2EFBC0945913742054185A53F82
:101DB000EF309071B777000083A5873DEF30E03AB0
:101DC000EF30707DB777000003A6073E83A6473E3D
:101DD000EF20803CB777000003A6874083A6C7406A
:101DE000EF20803BEF40E0056FE0CFBAEFE24FB865
:101DF0000D45ED3D420541853D37EF30F06CB7773D
:101E0000000083A5873DEF304036EF30D078B777BC
:101E1000000003A6073E83A6473EEF20E037B777D2
:101E2000000003A6873E83A6C73EEF20E0362A8641
:101E3000AE86EF10302DEF40C0006FE0AFB5EFE29F
:101E40002FB31145653542054185F13DEF30D0672F
:101E5000B777000083A5873DEF302031EF30B073B6
:101E6000B777000003A6073E83A6473EEF20C032A7
:101E7000B777000003A6074083A64740EF20C03194
:101E8000EF30307C6FE00FB1EFE28FAE1945B93D16
:101E900042054185493D9D67938707410147930668
:101EA000100F92236369C5023A85EF20506EB77711
:101EB000000003A6073F83A6473FEF20E02DB7773A
:101EC000000003A6873F83A6C73FEF206078EF306E
:101ED00050776FE02FAC05078907E314D7FC130593
:101EE0000000C5BFEFE2CFA8797148001306A00239
:101EF0008145EFF06FCE188293073005370500203B
:101F00006317F70298829307C0046312F70203472E
:101F1000D102D947631DF7001306A0024C00130538
:101F20000502EF40800F054545616FE0AFA6B7079A
:101F3000002003C7C704130505029387C70418A12F
:101F4000983318B1B82338A1B83338B1D82358A181
:101F5000D83358B1F82378A1F83378B19827DC3713
:101F600018A5A304F5020145C1B7EFE26FA0411126
:101F70002A8940000408029908C01104E31D94FE58
:101F80001244A2442285A685EF3040496354A00044
:101F900026C222C41244B2452285EF30204863593C
:101FA000A000A2452285EF30C04F6353050022C434
:101FB000224541016FE00F9EEFE2EF9941112AC6E1
:101FC000372500001305E5E34D37B245AA89EF3008
:101FD000407FB777000083A507659384C180EF3009
:101FE0000055B777000083A547642A894E85EF30F6
:101FF0000054AA854A85EF20B0608C40EF205060E5
:1020000088C01385C180EFF0CFE841016FE0EF9702
:10201000EFE26F9493878189F827C0372207418FB9
:10202000E0371389C1804204418F802B6204598CB0
:10203000A285EF300079B777000083A58764EF3081
:10204000004FB777000083A54764AA892285EF3047
:10205000004EAA854E85EF20B05A83250900EF2057
:10206000305A2320A9001385C180EFF08FE26FE082
:10207000CF91EFE24F8E93878189B82B803B220767
:10208000418FA03B1389C1804204418FC02B620461
:10209000598CA285EF30E072B777000083A5076501
:1020A000EF30E048B777000083A50764AA8922854E
:1020B000EF30E047AA854E85EF2090548325090034
:1020C000EF2010542320A9001385C180EFF06FDCAE
:1020D0006FE0AF8BEFE22F88138781898347470238
:1020E000834637021147A207D58FFD17C207C18368
:1020F0006360F7021D678A071307475FBA979C431F
:10210000138481898287B777000003A5076195371B
:102110006FE0AF87B777000003A54761713DCDBF82
:10212000B777000003A58761E535DDB71387018127
:102130001C239384018685C3B7060020938606027C
:10214000BC2E903E9306800CA207D18FB387D70296
:10215000230007009CC0371500408145130505800A
:10216000EFE0DFED9387C18598439440050798C35E
:10217000E310D7FA23A00700B777000003A5876113
:10218000413D8D47A301F4022302040251B7938419
:1021900011819C20138941858DC7B7070020938743
:1021A0000702E83B9C2FA2075D8DEF30F031B77737
:1021B000000083A5C760EF20507B2320A900238067
:1021C000040003250900377A000099357C24443443
:1021D000832A0900A207C58F6434D685C204C58F3F
:1021E0000428E204DD8C2685EF30A05DEF30B03AA4
:1021F00003290A6283294A624A86CE86EF109063D9
:102200006354A00228281C3822055D8D3C38C20783
:10221000C98F482862055D8DEF30F0374A86CE863B
:10222000EF10306C63420504A6855685EF30605987
:10223000EF30703603260A6283264A62EF10905F01
:10224000E358A0EC28281C383777000022055D8D64
:102250003C388325473BC207C98F482862055D8DFE
:10226000EF30C01BE356A0EAB777000003A5476133
:10227000EFF09FD4894739B7EFD21FED1389218141
:102280008347090093848185A5CB3704002013047C
:1022900004027C244834B7790000A2075D8DEF303A
:1022A000B02283A5C960EF20506C23A4A1841C2810
:1022B0006834A2075D8DEF30302183A5C960EF201F
:1022C000D06A23A6A1843C280838A2075D8DEF3090
:1022D000B01F83A5C960EF20506923A8A1847C2882
:1022E0004838A2075D8DEF30301E83A5C960EF200E
:1022F000D06788C023000900138781892C2F1C3FD9
:102300008840A205DD8D3C3F13848189C207CD8FB3
:102310004C2FE205DD8DEF3060106355A0087C285E
:10232000034954010438A207B3E7270103497401A4
:102330004209B367F9000349840162093369F9006E
:102340003C284A85A207C58F2438C204C58F44287B
:10235000E204DD8CA685EF30600C63520502CA856D
:102360002685EF300046EF301023B777000003A634
:10237000876283A6C762EF10D05663550502A3019A
:10238000040223020402EF007058B73500008146B2
:102390001306803E9385E50313854194EFF04FF1DA
:1023A0006FD01FDE7C244434A207C58F6434C2047E
:1023B000C58F0428E204DD8C03A9C1842685CA8563
:1023C000EF30C0056352A0022C281C38A205DD8D19
:1023D0003C38C207CD8F4C28E205DD8D03A5018571
:1023E000EF30C003634BA00083474402034734022D
:1023F000A207D98F11476398E7009147A301F40220
:102400002302040271BF03AA81842685EF30B0182D
:102410002A8B5285AE8BB7790000EF30D01703A618
:10242000096383A64963EF10E04D5A86DE86EF10FC
:10243000504B635405024A85EF30F01503A609633B
:1024400083A64963EF20C0202A86AE865A85DE85A2
:10245000EF1030498947E353A0FACA852685EF205B
:10246000F07B6355A00403A50185EF30D012B77748
:10247000000003A6076283A64762EF10A0482A89DE
:1024800028281C38AE8922055D8D3C38C207C98FCB
:10249000482862055D8DEF3010102A86AE864A8589
:1024A000CE85EF1010448D47E35AA0F4D2852685DF
:1024B000EF20307F8547E34305F43C2803491401AE
:1024C0004438A207B3E72701034934014209B3673F
:1024D000F9000349440162093369F9007C284A85FF
:1024E000A207C58F6438C204C58F042CE204DD8CBA
:1024F000A685EF30002DEF30100AB777000003AA51
:10250000876383AAC7635286D686EF10903DE3594E
:1025100005E8CA852685EF30C02AEF30D0075286FD
:10252000D686EF10103CE35D05E69547C1BDEFD2BE
:102530003FC437250000130525DAEFF01FA31384ED
:1025400081899357850048B47CA493570501618124
:1025500008A837250000130505D57CB4EFF0FFA0CF
:102560009357850008B83CA893570501618148A896
:10257000372500001305C5DE3CB8EFF01F9F9357C9
:1025800085007CA8935705017CB883C7118848B89B
:10259000618108AC99E3EFF03FCEEFF0BFB36FD0AD
:1025A0007FBFEFD2FFBC378500001306E0228545D0
:1025B00013058580EF3090319387818903C53702F9
:1025C00083C74702A2075D8D6FD0DFBCEFD25FBA31
:1025D0003775000013062022854513054579EF3035
:1025E000F02E03A5818B2181420541816FD09FBAD6
:1025F000EFD21FB83775000013066021854513051B
:10260000C57CEF30B02C93878189D84F03C5070272
:10261000B777000083A5877C21836205598DEF2061
:102620001071EF30A058420541816FD0BFB6EFD294
:102630003FB4378500001306A02085451305458368
:10264000EF30D02893878189984FC82FB777000043
:1026500083A5877C21836205598DEF20506DEF3073
:10266000E054420541816FD0FFB2EFD27FB03775A1
:1026700000001306E01F854513050576EF30102591
:1026800093878189D84B882FB777000083A5877CF3
:1026900021836205598DEF209069EF30205142056A
:1026A00041816FD03FAFEFD2BFAC3775000013064A
:1026B000201F854513050573EF30502193878189CD
:1026C000984BC82BB777000083A5877C21836205D0
:1026D000598DEF20D065EF30604D420541816FD0BC
:1026E0007FABEFD2FFA8377500001306601E85454B
:1026F0001305C56FEF30901D93878189D847882BCC
:10270000B777000083A5877C21836205598DEF2070
:102710001062EF30A049420541816FD0BFA7EFD2D0
:102720003FA5377500002E841306F0148545130568
:102730004565EF30B01905472381E1881385418F46
:1027400023820186EFF0AFBA5C245834B73500001D
:10275000A207D98F81461306803E9385A553138522
:102760004192239CF188EFF0AFB46FD0BFA2EFD2BB
:102770003FA023ACA18615470566B7350000238E20
:10278000E18685448146130686BB9385E53E138525
:10279000418F23829186EFF0AFB1238A918E6FD063
:1027A0007F9FEFD2FF9CD425DC35A206DD8E9547B6
:1027B00063FDD700377500001306401285451305E9
:1027C0000568EF30B0106FD0FF9CB425BC35A20671
:1027D000DD8E9307002063FAD700377500001306DB
:1027E000B01285451305056BE9BF37750000130569
:1027F000856EEF30F01EC1BFC16769768146FD1757
:1028000005061397060141836364B7003E85828005
:102810003307D5001823B98F214713F81700858394
:1028200063050800B18FC207C1837D17420741834A
:102830006DF78506F9B7EFD2BF9337150040130542
:102840000580EFE01F81EF30701AEF30901F930783
:10285000100F3365F502A94729053305F5026FD03E
:102860007F93EFD25F8F03A781882A84BE840546B9
:1028700093055052631CA70437550040130505808B
:10288000EFE0FF8D2285EF100007131905010945C0
:10289000EFF08FB62285EF10000683A78188931989
:1028A00005011359090193D90901014693055052B5
:1028B000375500406391870213050580EFE03F8A9A
:1028C000330539413335A0006FD03F8C3755004078
:1028D000130505C075B7130505C0CDB7EFD25F89E5
:1028E00037040020834704024111130404025C8072
:1028F0001C3023150100AA84DC803C20AD450A85EC
:102900005C813C3023160100DC815C205C825C3001
:10291000DC827C205C837C30DC831C245C84930719
:1029200010FDDC8485475C85EFF01FED9357850033
:10293000DC85834794024886DC86EFF0DFEFEFF01A
:10294000AFAB2685EFF0FFF16DF93D468A85268510
:10295000EF00B07083A78188054693055052375524
:1029600000406399970013050580EFE04FFF410198
:102970006FD05F82130505C0CDBFEFD26FFF370464
:102980000020834704024111130404025C801C30C0
:1029900023150100AA84DC803C20AD450A855C81BA
:1029A0003C3023160100DC815C205C825C30DC82E0
:1029B0007C205C837C30DC831C245C84930700FDDA
:1029C000DC8485475C85EFF03FE393578500DC8529
:1029D000834794024886DC86EFF0FFE5EFF0CFA155
:1029E0002685EFF01FE86DF93D468A852685EF00C4
:1029F000D06683A78188054693055052375500401D
:102A00006399970013050580EFE06FF541016FD0E2
:102A10006FF8130505C0CDBFEFD20FF303C9C50092
:102A2000DC35011122093369F900420913590941C2
:102A300093140901C180954763FF97003775000023
:102A4000A6861306500C854513050568EF3000680F
:102A500005616FD0EFF2B425BC35A206DD8E930779
:102A6000002063FAD700377500001306B00C8545C7
:102A70001305056BE1BFAA8902CA02CC231E01001F
:102A8000930A4101368A370B0020B307DA40C207A8
:102A9000C18363E1970C1384018C1305C4001306F2
:102AA00060028145EFD0CFEF370700208347070250
:102AB000A3052401230504001CA0930707029433F7
:102AC000939A14001309070214B0B42334A0B4334A
:102AD00034B0D42354A0D43354B0F42374A0F433CA
:102AE0009C2774B01CA4930700031CB48147138473
:102AF000C18C63C5570993856400860593F5E50F7E
:102B00001385018CEFF05FCF9317850021815D8DD8
:102B10008347990256940AA03CA0EFF0DFD1EFF072
:102B2000AF8D4E85EFF0FFD36DF913860A019385C3
:102B3000018C4E85EF00705283A78188054693056E
:102B4000505237550040639C370513050580EFE070
:102B50000FE1FDBD1304CB08930B84031C40639964
:102B600047015C40014536C68297B2462390AA00D1
:102B70002104E3958BFE890A050A01BF101013F7A3
:102B8000E70F329713F61700B306F400035747FF19
:102B900011E22183850798A293F7F70F99BF1305D8
:102BA00005C075B7EFD22FDB370400201304C4052E
:102BB000AA89AE84328A1309040398341C4063172F
:102BC000F7005C405286A6854E8582972104E31665
:102BD00024FF6FD08FDBEFD2AFD641112A8CEF00EC
:102BE000904D6308052A5145EFF00F81130620032D
:102BF00081451385018C1384018CB70D0020EFD023
:102C00002FDA81498144014A930B1400B78C0000EC
:102C1000378D0000138B0D026285EF00D04D630AE3
:102C200005266285EF00B04A9387018CD2973EC695
:102C300088A3930A1A0089476384FA00638E0424E8
:102C4000182083C70D026314F710183083471B0048
:102C5000631FF70E378500001306102785451305FF
:102C60000587EF30A046A5476394FA0603D781890C
:102C70008947631DF708382083472B00631BF7083B
:102C8000383083473B006316F708582083474B00D2
:102C90006311F708583083475B00631CF706782000
:102CA00083476B006317F706783083477B00631216
:102CB000F706182483478B00631DF704378500004F
:102CC0001306A02885451305C589EF30204021A0B3
:102CD0008547E3ED97F8A9476385FA00894763FFC5
:102CE000970883D78189094714346392E712130741
:102CF00000036399E606378500001306B02D85456D
:102D00001305C58FEF30803CC5498DA883C7418628
:102D1000BDF383C7418195CB38303C20F98F5820D3
:102D2000F98F5830F98F7820F98F7830F98F18247F
:102D3000F98F1307F00F639AE70037850000130639
:102D4000F02985451305858C49B791E08544528665
:102D5000DE851385018CEF30402C93070003E3FDE3
:102D600047EB05AA41476398E60237850000130642
:102D7000102E854513050592EF3040351834C147B4
:102D80006312F70CB54763FF570B8349D4008609DC
:102D9000C509568AD9B7138706031377F70F054677
:102DA000636DE600378500001306802E8545130508
:102DB0004594EF30A031B549D1B703C741811DCF4C
:102DC0001307000A1306E02E6389E6041307100AAE
:102DD0006398E6001306402F854513058D981DB7AF
:102DE000268763F3F40009479374F70F1306C02F87
:102DF000854513850C9BEF30602D91BF268763F3CB
:102E0000F40009479374F70F13067030D5B7930792
:102E1000000A639AF60013060031378500008545E5
:102E20001305459679B79307100A13066031E385B9
:102E3000F6FAA68763F3E400894793F4F70F1306C5
:102E4000E0317DB7E3973AF59385DAFF93F5F50F17
:102E50001385018CEFF05F9A330744018347E7FF46
:102E60000347F7FFA207D98F6397A700B2479823BC
:102E7000D947630AF7000D47A68763F3E4008D473F
:102E800093F4F70FE9B556869385018C6285EFF0D0
:102E90007FD141016FD08FAEA547E39EFAE2F9B32F
:102EA000EFD20FAD938741889843D5669386061875
:102EB0006307D702050798C33714014085649385DB
:102EC0000480130504800546EFD05FB20146938568
:102ED000048013050480EFD07FB16FD0AFAB23A087
:102EE0000700B707EFBE37E700E0938707083CC746
:102EF000E1B7EFD2EFA7B777000083A5C76403A5BA
:102F0000C18013848189EF208062EF201044AA855C
:102F1000378500001305459DEF30401B68245C3465
:102F2000B774000022055D8D7C3483A5C460C207A0
:102F3000C98F082862055D8DEF20605FEF20F040AB
:102F4000AA85378500001305C59EEF302018282874
:102F50001C3883A5C46022055D8D3C38C207C98F2B
:102F6000482862055D8DEF20805CEF20103EAA8529
:102F700037850000130505A0EF30401568285C3840
:102F800083A5C46022055D8D7C38C207C98F082CDB
:102F900062055D8DEF20A059EF20303BAA85378573
:102FA0000000130545A1EF306012682C5C3C3777B8
:102FB000000022055D8D7C3C8325877CC207C98F7C
:102FC0000345040262055D8DEF206056EF20F03767
:102FD000AA8537850000130585A2EF30200F8347AF
:102FE00024028345140237850000A207DD8D1305F6
:102FF00085A3EF30A00D8347440283453402378513
:103000000000A207DD8D1305C5A4EF30200C9387C7
:1030100041879023371501409305001013361600A1
:103020001305058090A3EFD07F9C6FD0AF96EFD2B1
:103030002F9403A5C188EFF01FBA6FD0AF95EFD2E0
:103040002F93B704002093870402D42FB83FA20621
:10305000D98E13873181102393840402938781864C
:1030600011C6230007001387D6FF9AA39A230507EA
:10307000420741836305D7009AA36FD0AF913725EC
:1030800000001305E5E32390070037790000EFE027
:10309000DFED138481898325C96013578500935719
:1030A000850138AC1357050138BC5CAC08BCEF2077
:1030B0000048EF209029AA8537850000130585AACE
:1030C000EF30C0003C2C183CA838A2075D8F3C3C78
:1030D000402CC207D98F62045D8CDC28A2075D8D6D
:1030E000EF20903E8325C960EF202008A285EF20C5
:1030F000403BE35405F8B735000081467946938597
:10310000C53313854193EFE0BF9A85BFEFD24F8659
:10311000371501400546A145130505C0EFD01F8DA9
:10312000378700000327C7AB3715004081451305DB
:10313000058023A6E180EFD07FF037050040814570
:1031400013050540EFD09FE86FD0CF84EFD2AF805A
:1031500013876186B7040020138604021E23742E91
:103160004C3E8507C207A206C183CD8E6385F6005B
:103170001EA36FD08F8137250000130525DA231099
:103180000700EFE09FDE138481899357850048B4E0
:103190007CA493570501618108A837250000130519
:1031A00005D57CB4EFE07FDC9357850008B83CA8D8
:1031B00093570501618148A8372500001305C5DE36
:1031C0003CB8EFE09FDA9357850048B87CA8935746
:1031D0000501618108AC37250000130585E87CB83E
:1031E000EFE0BFD89357850048BC7CAC371901404D
:1031F0009357050161812300A40293050010130574
:1032000009C07CBCEFD0AFFD93840402938981890F
:10321000814701C99145130509C0EFD0AFFBB33712
:10322000A000372500001305E5E3A380F902238100
:103230000902EFE09FD393578500238DF900935740
:103240000501A38DF90083C7E90103C7D901A38C48
:10325000A900A2075D8F618183C7F901238EA900B0
:1032600003C50902C207D98F62053369F50083C718
:10327000840203C57402A2075D8DEF209018AA8511
:103280004A85EF2000226356050283C6118809474C
:1032900013841188639CE600B735000081467946A7
:1032A0009385C53313854193EFE09F80230004008D
:1032B000C9B583C7640203C55402A2075D8DEF2020
:1032C0005014AA854A85EF206015635AA0009547DF
:1032D000A381F902054723820902A380E18883C7FD
:1032E000440203C53402A2075D8DEF209011AA8528
:1032F0004A85EF20A012E35EA0E60947A380E1889B
:10330000EFF0DFE0BDB5EFC2BFE6370500409387C1
:1033100081890947854513050540A381E70223827A
:103320000702EFD0BFCA37150140054693050010CC
:10333000130505C0EFD08FEB6FC0DFE5EFC2BFE133
:103340001387E1871E231384E1878507C207C183A2
:103350001EA30547639EE70037150140130505C00E
:103360000146A145EFD08FE813854194EFE02FF897
:103370001E201147636CF700371500409305400687
:1033800013050580EFD09FCB6FC03FE013076004AB
:103390009384C186636BF70083A9040083A5C18071
:1033A0004E85EF20A0076352A0029307000013850B
:1033B000C1809CC023100400EFE0AFAD13854193A2
:1033C000EFE0EFF2EFF03FF4C1B74E85EF20B01C15
:1033D000B787000003A607AA83A647AA2523EF20E4
:1033E000502688C01385C186EFE0AFAA71BFEFC237
:1033F0009FD6138731881C23011193861700F51778
:1034000014A393F7F70F9306B00F63EDF60013853F
:10341000418F2382018623000700EFE04FED056115
:103420006FC0BFD6414681451305E100EFC05FD7AD
:10343000370400208347040213040402DD455C8244
:103440001C30480093843188DC82FD577C83FD5713
:103450003EC4E9779387F71F7C8683C7C187DC87E3
:1034600003C7918983C68189938781892207558FF4
:10347000A308E1009356870038202308D1002309D0
:10348000E1003830A309E1005820230AE100583058
:10349000A30AE1007820230BE1007830A30BE100C0
:1034A0001824230CE1009837BC27A207D98F13D723
:1034B0008700230DF100A30CE100EFF0EFB3935769
:1034C0008500A30DF10083479402230EA100294437
:1034D000A30EF100EFF02FB6EFE00FF21389818712
:1034E00003250900EFF0EFB721E5938721889423A6
:1034F00005476397E600238007002380040005B793
:10350000032509006D464C00892E0327090083A777
:103510008188054693055052375500406317F700E0
:1035200013050580EFD0BFC3DDBD130505C0DDBFAA
:103530007D141374F40F59FCDDB593870187904314
:10354000938641810506B705002090C323800600BD
:103550009385050203C7250203C515022207498F7B
:10356000631EE600EFC2DFC023A00700138541926F
:1035700085479CA2EFE0AFD76FC0DFC18280EFC26A
:103580003FBFB707002093870702B82313848189C0
:1035900038A0B833238C0188A38C018838B0D82395
:1035A00037250000130525DA58A0D8339384818984
:1035B00058B0F82378A0F8339C2778B0370700205C
:1035C0001307C7041CA43C271437A207D58F1CB4CB
:1035D000A1833CA45C273437A207D58F3CB4A183D8
:1035E0005CA4EFE09F989357850048B47CA4935760
:1035F0000501618108A837250000130505D57CB4B5
:10360000EFE0BF969357850008B83CA89357050193
:10361000618148A8372500001305C5DE3CB8EFE0FE
:10362000DF949357850048B87CA8935705016181C2
:1036300008AC372500001305E5E37CB8EFE0FF9206
:103640009357850008BC3CAC93570501618148AC99
:1036500037250000130585E83CBCEFE01F91935728
:10366000850048BC7CAC9357050161817CBC23007C
:10367000A4023714014093050010130504C0EFD0D5
:103680000FB6814701C99145130504C0EFD08FB42F
:10369000B337A000A380F40223810402A3810402B3
:1036A000238204026FC01FAFEFC29FACEFE09F8385
:1036B000EFF0FFECB735000081461306803E93859E
:1036C00025EF13854191EFE0AFBEB735000081468D
:1036D000130640069385E50213854195EFE04FBD43
:1036E000B7350000F9461306803E938505EA138539
:1036F0004196EFE0EFBBB73500009306803E13061E
:10370000803E9385C51413854190EFE06FBAB735BD
:10371000000081461306803E9385E503138541949E
:10372000EFE00FB9EFE08FBF6FC0DFA6EFC25FA47D
:103730000545EFE06FAE8D28EFD0FFEEEFD0FFAA8A
:10374000EFD01FD0EFD0BFD2EFD03FB9EFD05FD5D1
:10375000EFD0FFD8EFD01FE50545EFE0EFA06FC039
:103760007FA3EFC2FFA0014405C1002111CC5C4141
:103770000D47639EE7003755004093F5F50F13059D
:103780000580EFE0EF8E054422856FC0BFA0114792
:103790000544E39BE7FE3755004093F5F50F13050D
:1037A00005C0EFE0EF8CCDB7EFC29F9C370400203F
:1037B0001304440C1306800C938541971305C40031
:1037C000EFE06FBA08448544EFD0BFFE04A01306B3
:1037D000C0129385C1A31305840223A48188EFE05E
:1037E0008FB848507104EFD0BFF104A0014523A663
:1037F00081886FC03F9AEFC2BF97371501400546D9
:1038000093050002130505C0EFD04F9E6FC09F982F
:10381000EFC21F96371501400146930500021305BC
:1038200005C0EFD0AF9C6FC0FF96EFC27F943715F5
:1038300001400546C145130505C0EFD02F9B6FC061
:103840007F95EFC2FF92371501400146C145130530
:1038500005C0EFD0AF996FC0FF93EFC2DF8F03A712
:1038600081882A842E8AB28993848188631EA70066
:10387000EFF07FF80149634039039C40639687026B
:10388000EFF01FF96FC07F9083A7C188E394A7FE74
:10389000EFF0BFF9C5B7B3072A018385070022857A
:1038A0000509EFF01FECC1BF83A7C188E39C87FC2B
:1038B000EFF03FF9C1BF814709C91821814711C7FE
:1038C0005C49084D898FB337F0003E858280EFC296
:1038D0003F8A41112A84A3070100EFF0DFFD19C5DB
:1038E0009305F1001305C400EFE0AFAB0305F10051
:1038F00041016FC03F8AEFC2BF873105EFE0CFAC17
:103900006FC05F893708100001117D183377B80048
:1039100026CA3378D80093D4450113D34601131E29
:1039200037004EC61357D5010E089357D60193F4AE
:10393000F47F1373F37F06CE22CC4AC893D9F501E6
:1039400093DEF6013367C701131F350033E8070123
:10395000931F3600338E64406380D9196356C013B9
:103960006304031CB70680009307F07F3368D80018
:10397000638FF4369307800363C0C735FD4763CD7B
:10398000C747130500023305C541B3D7CF01B316AE
:10399000A8003399AF00DD8E33392001B357C80139
:1039A00033E926011D8F33092F41B3372F01330629
:1039B000F7409317860063D40724370780007D17EC
:1039C0003374E600630C042C2285EF20205E13077D
:1039D00085FF93070002998FB357F9003316E4006F
:1039E000D18F3319E9006341972A330597401306B5
:1039F00015007D47634DC73813070002118FB3567A
:103A0000C9003319E9003397E700558F3339200196
:103A10003369270133D6C70081449377790081CF7A
:103A20001377F90091476308F7001307490033390A
:103A300027014A963A899317860063D6071C138597
:103A400014009307F07FCE856304F520B70780FF4D
:103A5000FD17F18F9398D70113593900A607B3E8E2
:103A60002801B1831375F57F9396C7005205F24084
:103A70006244B182FE05C98ECD8ED2444249B2491C
:103A80004685B68505618280631E0E0A1383140085
:103A90001373E37F63170322B367E701B368F80189
:103AA000639D041A63870740638608443309FF4116
:103AB000B307074133362F013386C740931786007B
:103AC00063D6074C3389EF41B307E84033B62F0183
:103AD0003386C740F68991B76350C00F6300030C6B
:103AE000B70680009307F07F3368D800638AF43A02
:103AF0009307800363CBC713FD4763DFC735130903
:103B00000EFE93070002B3562801630AFE00130954
:103B100000043309C94133192801B3EF2F013339A8
:103B2000F0013369D90031A2B367F801638A071C39
:103B30009307FEFF638C07389306F07F6309DE1A54
:103B40003E8E0DBDB305934063910422B367E70138
:103B5000638707329387F5FF638107449306F07FFD
:103B6000638CD520BE859307800363CCB72AFD47BD
:103B700063CFB73C930700028D8F3319F700B3561C
:103B8000BF00B317FF003369D900B337F0003357D4
:103B9000B7003369F9003308E84041ACB367F80176
:103BA000638007349307FEFF638A07209306F07F44
:103BB0006308DE2E3E8E2DBF631E0E149386140006
:103BC00093F7E67F63910734B367E7016395042CAD
:103BD0006380073EB367F801638E07303309FF0146
:103BE000B3070701333FE9013386E70193178600E6
:103BF00063D70700B70780FFFD177D8E8544937755
:103C00007900E39F07E09317D60193583900B3E892
:103C1000F800935736001307F07F638DE404B20772
:103C2000B18313F5F47FCE8581B53369F80133395B
:103C300020017A99B337E9013386E70093178600AC
:103C4000E3DF07FA85049307F07F6396F418CE85C7
:103C50001305F07F8147814801BDC1EB6384083AB9
:103C6000931636009317D8018D82B3E8D700F689F2
:103C700093573800B3E7F800F9DB81451305F07F6F
:103C8000B70708008148CDB3370680FF7D167D8ECB
:103C900093777900998CE39507D8B5B74A85EF20DB
:103CA000E03013078501FD47E3D5E7D2130685FF12
:103CB000B317C900014905BB3369F8013339200145
:103CC000DDB13309FF413306074133342F0133049B
:103CD00086409317840063CD0724B3688900E3937B
:103CE00008CE8147814981441DBFE39808F80E053D
:103CF0009317D7010D81B3E8A700935737009DBFF5
:103D00000E059317D7010D81B3E8A700F2849357EE
:103D1000370011B73305934063820412B706800061
:103D20009307F07F558F630DF32E9307800363CBCA
:103D3000A720FD4763C3A72A93070002898F331981
:103D4000F700B356AF00B317FF003369D900B3379C
:103D5000F0003357A7003369F9003A987E99B337DA
:103D6000F901338607019A84D1BDB7068000930715
:103D7000F07F558FE319F3DE931736008D83931888
:103D8000D801B3E81701F68993573800E5B5130752
:103D900015FE9306000233D7E700630AD6009306A8
:103DA00000043386C6403396C7003369C9003339EF
:103DB00020013369E9000146814491B53309FF01CF
:103DC000B30707013336E9013E9693178600854411
:103DD000E3D707E28944B70780FFFD17F18F135738
:103DE000190013791900336927019398F70133E912
:103DF000280113D6170015B113090EFE9307000210
:103E0000B3562801630AFE00130900043309C941AF
:103E100033192801B3EF2F013339F0013369D90089
:103E200059B63369E7013339200133892F41B3B7DC
:103E30002F013306F8409A84F689A5BEB367E701DF
:103E4000638207189307F5FF6384071C9306F07FCE
:103E50006304D5123E85D1BD93070002B387C741E5
:103E6000B316F8003399FF0033D6CF01D18E333922
:103E70002001B357C80133E926013E975DBB931774
:103E800036008D839318D801B3E81701AE84935799
:103E90003800F68949B3EDC33369F801E31F09DC43
:103EA0000E059317D7010D81B368F50093573700BE
:103EB000D1B36381080E931636009317D8018D8213
:103EC000B3E8D700F6899357380091BB3309FF4117
:103ED000B3070741333F2F013386E7418544D1BC07
:103EE0000E059317D7010D81B368F500F28493573F
:103EF000370015B30E059317D7010D81B3E8A7005E
:103F00009357370029BB9307F07FE382F6D4330938
:103F1000FF013336E901B3070701B2979398F70120
:103F20001359190033E9280113D61700B684C1B913
:103F30003389EF413307E84033B62F013304C740DC
:103F4000F68949B43369E7013339200101BD93870C
:103F500005FE93060002B357F700638AD500930667
:103F60000004B385B6403317B700336FEF00333921
:103F7000E0013369F90055BD931736008D8393181E
:103F8000D801B3E8170193573800EDB1B368C90001
:103F9000E39708C68147814959B13389EF41B30797
:103FA000E84033B62F013386C740F689854411B403
:103FB000931636009317D8018D82B3E8D700935734
:103FC0003800B1B9931636009317D8018D82B3E843
:103FD000D700AA84935738003DB9930705FE93068E
:103FE0000002B357F700630AD50093060004338537
:103FF000A6403317A700336FEF003339E001336970
:10400000F900A9BB81451305F07FB7070800A9BCDB
:104010003309FF01B30707013336F9013E9675B343
:10402000931636009317D8018D82B3E8D7009357C3
:10403000380089B113D74501B7071000FD1713D811
:1040400046011377F77F9308F07F33F3B7002A8E8A
:10405000F58FFD81B28E1378F87FFD826308170318
:10406000630018030DEBB368A300631408005D8EB2
:1040700029CA638508046388D502054595ED8280C9
:10408000B3E8C700E38008FE795582803365A3005A
:1040900065FD630CE802631408005D8E79DEE39E23
:1040A000D5FCE34CE8FC63480701E3E867FC6303E5
:1040B000F302637FF30081E57D558280F5DE0545DF
:1040C00082800145E39B08FA82805D8E69DA6DBFCC
:1040D00001458280E3E3CEFB0145E372DEFBE5F1BF
:1040E000E1BF13D74501B7071000FD1713D84601EC
:1040F0001377F77F9308F07F33FEB700AA8EF58F12
:10410000FD81328F1378F87FFD82630E1703630DF4
:10411000180129E3B368AE00631F08005D8E01EE4D
:104120000143638C080421A8B3E8C70009436396E0
:1041300008046DD305A0638408046385D502054394
:104140008DCD7D531DA8B368AE0009436397080267
:10415000630AE802631408005D8E75D2E391D5FE10
:10416000E34FE8FC63490701E3EBC7FD630FFE0083
:1041700001436374FE00F1D505431A858280EDFE8C
:104180007D53E5BF5D8E79DACDBFE36ADFFB014386
:10419000E3F5EEFFF5F175B739714AD813D945014A
:1041A0004ED652D456D29399C50006DE22DC26DACA
:1041B0005AD05ECE1379F97F2A8A93D9C90093DA4F
:1041C000F501630D090E9307F07F6306F918135488
:1041D000D5018E09B36934013704800033E48900C6
:1041E00093143500130919C08149814B13D7460137
:1041F000139AC6001377F77FB285135ACA0013DBF0
:10420000F601630B07109307F07F6303F7049357DE
:10421000D6010E0A33EA4701130717C0B70780001B
:10422000B367FA00931536003A99814833C76A019B
:10423000BD463A851308190063E836171746000093
:10424000130646888A09B29983A60900B296828627
:10425000B367CA001309F97F6399071293E929002C
:1042600081458948E1B701479307F07F370408008B
:1042700081443204D20731807E075D8C598CA2853F
:10428000F250625426854259D254B259225A925A57
:10429000025BF24B216182805A853E84AE84C68BDC
:1042A0008947638DFB0E8D47E38FFBFA85472A878D
:1042B000639EFB3881470144814465BF33E4A90014
:1042C00061C036C632C4638C092A4E85EF10104E89
:1042D0002246B246AA87130755FF7544938487FF89
:1042E000198CB399990033548A0033643401B314A0
:1042F0009A0013D746011309D0C0139AC60013774A
:10430000F77F3309F9408149814BB285135ACA00BE
:1043100013DBF601E31907EEB367CA00B1C7630FF9
:104320000A22528532C4EF10704822462A8793062B
:1043300055FFF547930587FF958F331ABA00B3579A
:10434000F600B3E74701B315B6003309E940130996
:10435000D9C08148E1BD33E4A90001ECA149814401
:104360001309F07F894B59B593E9190081458548B8
:1043700075BD4E84AA84B1491309F07F8D4BBDB53C
:10438000914981440149854B95B593E93900D2871C
:104390008D4869BD89475685E397FBF02A879307C7
:1043A000F07F01448144F1B5C16E1386FEFF93D6C0
:1043B000040113DE0501F18CF18D33869502338300
:1043C000B6029358060133059E021A95AA98B38245
:1043D000C60363F36800F692C16F1383FFFF33F5E2
:1043E000670093D30701B3F76800C2073373660011
:1043F0003E933306950293D80801B387A602135F54
:104400000601B3849302BE94FA94B38E760263F3EA
:10441000F400FE9E416A9307FAFF935F0401B376AE
:10442000F400B3F9F4007D8EC1803384D502C20953
:10443000338FD401B299CE98B307DE02935E0401A4
:10444000B385BF02AE97BE9E330EFE0363F3BE007C
:10445000529EC1679385F7FF33F6BE006D8C42060E
:10446000229693DE0E01B305D502769E3385AF0208
:1044700013D40501B386D302AA96A296B38FF30391
:1044800063F3A600BE9F41657D15B3F7A600C20782
:104490006D8DAA97B3855800B3B93501FA97B295D7
:1044A0003384370133B6C500B30EC4013385CE0063
:1044B00033343401B3B7E701C18F33BECE0113D417
:1044C00006013336C5003E943366CE0093949500C2
:1044D00032947E94B3E46400260493567501B33499
:1044E0009000DD8193179500CD8C558CDD8C931752
:1044F000740063DB070093D7140085889316F401DA
:10450000DD8CD58C058042899307F93F6359F0080B
:1045100093F6740081CE93F6F40011466388C600CA
:1045200093864400B3B496002694B6849316740020
:1045300063D80600B70700FFFD177D8C930709407D
:104540009306E07F63CFF60E93D634009314D40124
:104550002604D58C318093F7F77F21BB328532C496
:10456000EF10D02493065501F147130705022246A8
:10457000E3D1D7DC6115B317A6008145F9B3EF107D
:10458000F02213075501F145930705022246B24672
:10459000E3D5E5D461153314AA00814499BB85465F
:1045A0009D8EB1E71309E941B3972401B3D4D40038
:1045B00033192401B337F000B3649900DD8C93F70D
:1045C0007400B356D40081CF93F7F400114663888A
:1045D000C70093874400B3B49700A696BE84939710
:1045E000860063D8070485470144814459B1130606
:1045F0008003E341D6CC7D46E356D6FA0556B30791
:10460000F640930500023356F4006387B6001309A1
:10461000E943B3172401DD8CB3349000D18C93F6B9
:104620007400014499CA93F7F40011468146E3925D
:10463000C7FA139496003180F6068D80D58C814799
:104640000DB99307F07F0144814425B142896DBDC6
:10465000370710007D1701113373B70093D8460157
:10466000758F935ED60122CC26CA0E0393D44501E2
:104670009357D5010E0706CE4AC84EC693F8F87F69
:10468000130EF07F33E7EE0093F4F47F13D4F501BB
:1046900033E36700131F3500FD82931E36006380ED
:1046A000C81993C61600B38514416305D41263512B
:1046B000B018638B081AB70780005D8F6381C459F7
:1046C0009307800363C4B734FD4763C5B7489307B6
:1046D00000028D8FB3D9BE003318F700B39EFE00E1
:1046E000336838013357B700B339D0013368380124
:1046F0003303E340B3090F41B3373F013306F340BF
:104700009317860063D30724370980007D19337916
:104710002601630F092C4A85EF105009130785FF06
:1047200093070002998FB3D7F9003316E900D18FB0
:10473000B399E9006344972A058F13061700FD46D5
:1047400063C5C63A13070002118FB3D6C900339868
:10475000E9003397E700558F33380001B36907014B
:1047600033D6C700814493F7790081CF93F6F900DF
:1047700091476388F6009386490033B83601429624
:10478000B6899317860063D6071C13871400930716
:10479000F07F05886306F720B70780FFFD17F18FCC
:1047A0001398D70193D93900A60733683801B1832C
:1047B0001377F77F9396C7005207B1827E04D98E94
:1047C000C18EF2406244D2444249B2494285B68524
:1047D000056182806356B00A638A0812B7078000B9
:1047E0005D8F6387C42D9307800363C7B718FD47A8
:1047F00063D2B73C138805FE93070002B359070143
:10480000638AF50093070004B385B7403317B700F8
:10481000B3EEEE003338D0013368380195A2B367A8
:10482000D7019385148099E393C61600630AD404D4
:10483000D1E19387140093F7E77F6399071EB3676D
:10484000E3013368D701639204166382073C631661
:104850000842131835009316D3011358380033E873
:1048600006019357330019A2B367D7016385071A6E
:104870009387F5FF638B073A638CC523BE8589B5A3
:104880006399051C9386140093F7E67FC1EFB36725
:10489000E30163900436638D0744B367D7016394E3
:1048A00007460E051318D3010D813368A8009357EE
:1048B00033006DA8B385984063970420B367E30184
:1048C000638D07309387F5FF638907401305F07FF9
:1048D0006383A520BE859307800363C2B72AFD4783
:1048E00063C8B73C930700028D8F3318F30033562B
:1048F000BF00B317FF003368C800B339F00033536B
:10490000B3003368380133076740B5ACB367D701EC
:10491000638307109387F5FF638F071E6380C52F9E
:10492000BE85D1B59307F07F638BF606FA9E33B64A
:10493000EE01B307E300B2971398F70193DE1E0070
:10494000B369D80113D61700B68493F77900E39FB3
:1049500007E09317D60113D839003368F800A6850D
:10496000935736001307F07F6380E506B207B183E3
:1049700013F7F57F05883DBD3367D7013338E00075
:10498000B309E801B3B7E9013386670093178600DE
:10499000E3DD07FA85049307F07F639CF41805882C
:1049A0001307F07F8147014831B563910710630118
:1049B000083C131836009317D70113583800336892
:1049C000F800368493573700B367F800E9DB0144F9
:1049D0001307F07FB70708000148E9BB370680FFDF
:1049E0007D167D8E93F77900998CE39107D895B762
:1049F0004E85EF10A05B13078501FD47E3D2E7D298
:104A0000130685FFB397C90081492DB33368D701D9
:104A100033380001C5B1131835009317D30113586B
:104A200038003368F800935733002DBFB309DF41D6
:104A30003309E34033363F013309C94093178900F6
:104A400063CA072033E82901E31508CC81470144F4
:104A500031BFB385984063810414B7068000930783
:104A6000F07F3363D3006381F8209307800363CC26
:104A7000B722FD4763C9B72C930700028D8F331807
:104A8000F300B356BF00B317FF003368D800B33943
:104A9000F0003353B300336838011A97B309D801D3
:104AA000B3B7D9013386E700C684CDB5E31108F268
:104AB000131835009317D301135838003368F800E2
:104AC0009357330011B7370580009307F07F3363A6
:104AD000A300E392F8E00E061318D7010D823368A5
:104AE000C800935737003684C5B5051793060002F2
:104AF00033D7E700630AD600930600043386C64026
:104B00003396C700B3E9C90033383001B369E80010
:104B1000014681441DBDB309DF01B307E30033BF84
:104B2000E9013386E701931786008544E3DF07E058
:104B30008944B70780FFFD17F18F13D7190013F8C9
:104B40001900336807019399F701B3E9090113D6F6
:104B5000170011B9138805FE93070002B359070126
:104B6000638AF50093070004B385B7403317B70095
:104B7000B3EEEE003338D00133683801A5BE33639D
:104B8000E30133386000B3890E41B3B73E01330609
:104B9000F740C6843684ADB6B367E3016387071870
:104BA0009387F5FF638C071C9306F07F638ED50A0D
:104BB000BE8565BD930700028D8FB3D9BE00331843
:104BC000F700B39EFE00336838013357B700B3399E
:104BD000D001336838013A9365B313183600931740
:104BE000D7011358380033E807013684935737004C
:104BF00095BBBDCB3367D701E31B07DC0E0513184C
:104C0000D3010D813368A8009357330075BBE30FC0
:104C100008E2131836009317D70113583800336889
:104C2000F80036849357370091B3B309DF41B307D7
:104C3000E340333F3F013386E7418544D1B4131845
:104C400035009316D3011358380033E80601935703
:104C500033009DBBB389EE413306674033B93E0153
:104C600033092641368475B40E061318D7010D8218
:104C70003368C8009357370081BBB309DF41B307DE
:104C8000E34033363F013386C7409317860063D72E
:104C9000070AB389EE41B3076740B3BE3E013386CE
:104CA000D7413684C9B43363E30133386000FDB3C0
:104CB000138805FE93070002B3590301638AF500C8
:104CC00093070004B385B7403313B300336F6F000D
:104CD0003338E001336838017DB5B389EE41B3075D
:104CE0006740B3BE3E013386D7413684854409BC54
:104CF000131836009317D701135838003368F8009B
:104D000093573700A5B1B309DF01B307E30033BF01
:104D1000E9013386E70193178600E3D807C2B70796
:104D200080FFFD177D8E85440DB10E061318D70147
:104D30000D823368C800935737002DB133E8C9009E
:104D4000E30608D019B1138805FE93070002B35992
:104D50000301638AF50093070004B385B74033135A
:104D6000B300336F6F003338E001336838013DB36F
:104D700001441307F07FB70708002DBCB309DF011A
:104D8000B307E300B3BED9013386D70169BB411134
:104D900006C622C426C20DCD9357F541B3C4A70061
:104DA0009D8C2A842685EF1060209306E041898E31
:104DB000A9477D8093F6F67F63CDA7022D47098F23
:104DC000B3D7E4005505B207B394A400B18329A07A
:104DD0000144814681478144B207D206B1837E04F3
:104DE000D58FC18FB24022442685BE8592444101B1
:104DF00082805515B397A400B207B1838144E9BFFF
:104E00004111370780007D1713D8750126C29354CE
:104E100075013373A70093F4F40FB376B7004AC05B
:104E20001378F80F1359F50106C622C4FD819A873D
:104E300026854A86131E3300939E3600B3880441AC
:104E4000630AB90E6350100D630408149307F00F42
:104E5000638BF414B7070004B3EEFE00ED4763C1A3
:104E6000172993070002B3871741B397FE00B3D801
:104E70001E01B337F000B3E7F800B307FE40139705
:104E80005700635E0718370400047D147D8C22856B
:104E9000EF10C0116D15B317A4006348951A058D66
:104EA0001304150013070002018F3397E70033370F
:104EB000E000B3D78700D98F814413F7770019C773
:104EC00013F7F70091466303D70091071397570034
:104ED000635B071485041307F00F4A866383E416A7
:104EE0009A07A58313F5F40FB2402244A607931442
:104EF000750113D59700458D7E0692440249518D68
:104F0000410182806399080A138714001377E70F21
:104F10006317071463900422630D0E1EE3860EFCD4
:104F2000B307DE411397570063500722B387CE4182
:104F30002E8961B7635C100B630E08089307F00FAE
:104F40006383F406B7070004B3EEFE00ED4763C9C0
:104F5000171F93070002B3871741B397FE00B3D81A
:104F60001E01B337F000B3E7F800F297139757002C
:104F70006357070A85041307F00F6384E40CB70630
:104F8000007E13D71700FD16858B758FD98F35B727
:104F9000638D0E08FD18B307DE41E38208EE930728
:104FA000F00FE39DF4EA630D030801461305F00FCB
:104FB000B707400015BF33079840EDE863020E14B1
:104FC0007D17630807189307F00F6319F80E2E89F1
:104FD0003683D1BF638B0E04FD18B307DE01E38770
:104FE00008F89307F00FE393F4F675BF639508088C
:104FF000850413F7E40F6313071263170510630F9B
:105000000E14E3830EEEB307DE01139757008144BD
:1050100063570700370700FC7D17F98F854413F7A6
:105020007700E31F07E813D337009307F00FE38CF3
:10503000F4F693179300A58313F5F40F4A866DB524
:105040004A861305F00F814745B5370700FC7D17E9
:10505000F98F13F77700898CE31407E6E9B7330477
:10506000DE419317540063C3070CE31204E20146C8
:105070000145814795BD33079840ADC49307F00FB4
:10508000E308F8F4B7070004336EFE00ED4763CC85
:10509000E70C93070002998FB317FE003357EE0019
:1050A000B337F000D98FF697C284C9B59307F00FD4
:1050B000E30FF8F0B7070004336EFE00ED4763C35B
:1050C000E70893060002998EB316DE00B357EE0090
:1050D0003337D000D98FB387FE40C2842E8945B3C1
:1050E000854761BB630E0E067D17B307DE01C284E0
:1050F000E30E07E69307F00FE31AF8F8368365B579
:105100003683C2842E8915B7E3040EECE38D0EE8D6
:1051100069BD638D0E022E86B687F9B39307F00F33
:10512000E381F4F2B307DE018583D5BD3384CE413C
:105130002E89B1BBE31C0EFCE3890EE62E8949BD26
:10514000854725B5854741BFE39B07EC014681476D
:1051500061BBB387CE41C2842E8915B3B68769B3CC
:105160003683C284D9B585473DBF397193577501E0
:105170004AD856D25ECE931A95001359F50106DE31
:1051800022DC26DA4ED652D45AD093F7F70F93DAB0
:105190009A00CA8B638207121307F00F6384E71229
:1051A0008E0A37070004B3EAEA00138A17F80144AD
:1051B000014B93D775019394950093F7F70FA58052
:1051C00093D9F501FDC71307F00F6387E7028E043B
:1051D000938717F837070004D98C330AFA408146C1
:1051E000558C173700001307E7910A043A941C40C6
:1051F00033493901BA978287130A1AF0F9E88946C8
:10520000558C173700001307E7930A043A941C40A3
:1052100033493901BA97828701491307F00FB7075D
:10522000400013959700F25062549317770125813F
:105230007E095D8D33652501D2544259B259225AF7
:10524000925A025BF24B216182801307F00F814773
:10525000C9BFA68ACE8B368B8947630BFB1A8D4755
:10526000E30CFBFA8547630AFB0A1307FA0713F9F5
:105270001B006357E01293F77A0099C793F7FA007F
:1052800091466383D700910A93974A0063D9070038
:10529000B70700F8FD17B3FAFA0013070A089307D7
:1052A000E00FE3C4E7FA93976A00A5831377F70F3B
:1052B0008DBFB9E48546A9B763940A021144014A37
:1052C000054BC5BD63990A002144130AF00F094B31
:1052D000CDB58D4631B73144130AF00F0D4BD1BD1A
:1052E00056852EC6EF00904C9307B5FFB39AFA008F
:1052F0009307A0F8338AA7400144014BB24555BD3E
:105300002685EF00B04A1307B5FFB307AA00B39490
:10531000E400138A67078146E1B513F91B000147D2
:10532000814701B74166139554007D1693570501D7
:10533000698E63FA9A0AB3D5FA027D1AD6860147B6
:105340003388C502B3F6F602C206558F637B0701A8
:105350002A979386F5FF6368A70A6376070BF9150A
:105360002A9733070741B356F7023377F702B38A18
:10537000C6029317070163FB5701AA971387F6FF2D
:1053800063E1A70863FF5707F916AA97C205B38A16
:105390005741D58DB33A5001B3EA5501CA8BF1B5E7
:1053A0008546998E11C76D4601478147E34BD6E686
:1053B000130AEA09339A4A01B3D7DA00B33A400133
:1053C000B3E7570113F7770019C713F7F7009146B2
:1053D0006303D700910713975700634807029A07A2
:1053E000A58301473DBD93D61A00B3D5F6021397A6
:1053F000FA0141833388C502B1B7CE8B368B814A1F
:10540000A1BDBA8661B7B685A9BF0547814711BD61
:1054100013F91B001307F00F814721B5935675014F
:10542000B7078000FD1713D6750193F6F60F130822
:10543000F00FB3F8A7001357F501ED8F1376F60FB1
:10544000FD8163810603630C06018DE211E2B1C3A5
:10545000638E08026305B70405451DE78280F5D712
:1054600079558280E39E08FE6309D60211E2EDD7EA
:10547000E314B7FEE342D6FE63C7C600E3EE17FDB2
:105480000145E3FDF8FC01E77D558280F5DD05452A
:1054900082800145E39208FC8280F9DBD1B7814626
:1054A000E1BF93567501B7078000FD1713D675014C
:1054B00093F6F60F1308F00FB3F8A7001357F50192
:1054C000ED8F1376F60FFD816387060363090601EE
:1054D00085EA11EA89EB0145639B08008280094552
:1054E000F5FFE5DA31A8638C08026300B7040545CF
:1054F00075D77D5582800945639808026304D602FA
:1055000011E2F5D7E315B7FEE343D6FE63C7C60045
:10551000E3EF17FD0145E3F3F8FC19E3D9BFF1D937
:1055200005458280E5D3828082808146C5B7797146
:1055300022D4135475014ECE52CC9319950006D641
:1055400026D24AD056CA5AC81374F40F93D9990078
:10555000135AF50169C49307F00F6308F40E93978B
:10556000390037070004B3E9E700130414F8814455
:10557000014B13D77501939A95001377F70F93DAC0
:105580009A0013D9F50145CF9307F00F630CF7028A
:105590008E0A130717F8B7070004B3EAFA003A9423
:1055A000014633452A01BD47AA869305140063E2EC
:1055B0009710172700001307E75C8A04BA949C40F1
:1055C000BA9782871304F40F63980A0C93E42400BB
:1055D0000946C1BF01451307F00FB7074000B2509D
:1055E0002254A6075E07A5837E05D98F92540259DF
:1055F000F249624AD24A424B5D8D45618280CA8639
:10560000D689328B89476301FB0A8D47E304FBFC93
:10561000854736856312FB1A01478147C9B7639EE8
:10562000090413D77501939A95001377F70F9144E6
:105630000144054B93DA9A0013D9F50131F7639DC4
:105640000A0093E414000546A9BF63930902A1442C
:105650001304F00F094B31BF5685EF003015930747
:10566000B5FF098CB39AFA001304A4F8014615BFDC
:10567000B1441304F00F0D4BEDBD4E852EC6EF0067
:10568000F0129307B5FF1304A0F8B399F900098C41
:105690008144014BB245F1BD93E434000D4611B78E
:1056A0008947D286E313FBF636851307F00F81474F
:1056B0003DB741639306F3FF13D6090193D80A015E
:1056C000B3F7D900B3FADA0033885703B389F80285
:1056D00013570801B30A5603D6994E97330616039B
:1056E000637357011A96C167FD17B376F7003378D5
:1056F000F800C206C2969399660093570701B33922
:105700003001E982B2979A07B3E6D900B3E9D7002E
:105710009397490063D9070013D7190093F719002D
:10572000B369F7002E841307F4076350E00493F77E
:10573000790099C793F7F90091466383D7009109DF
:105740009397490063D90700B70700F8FD17B3F92D
:10575000F900130704089307E00F63CBE70493975E
:105760006900A5831377F70F9DBD8547B386E74092
:1057700011C76D4601478147E343D6E61307E409A5
:105780003397E9003337E000B3D7D900D98F13F747
:10579000770019C713F7F70091466303D700910705
:1057A00013975700634C07009A07A583014705BD6F
:1057B0001307F00F814725B52E84B5B705478147FC
:1057C00039BD3707800041117D179356750113D8F5
:1057D0007501B377A70093F6F60F935EF501337664
:1057E000B70026C24AC01378F80F06C622C41303B6
:1057F000F00F3E8E3689F684139F3700FD81131516
:105800003600B38806416302681093C51500638CA7
:10581000BE106354100D631008106304051EFD18BC
:10582000B307AF40638608029307F00F6388F6164C
:10583000ED4763C7172913070002330717413317D2
:10584000E500B35715013337E000D98FB307FF40A8
:10585000139757006351071A370400047D147D8C99
:105860002285A9276D15B317A400634E251B3305A8
:1058700025411304150013070002018F3397E70039
:105880003337E000B3D78700D98F014913F777008A
:1058900019C713F7F70091466303D70091071397D1
:1058A0005700635E0714930619001307F00F93FE69
:1058B00014006386E6169A07A58393F6F60FA607EB
:1058C000B240224413D59700DE069397FE01558D12
:1058D000924402495D8D410182806392080A1387D8
:1058E00016001377E70F631B071463940622630205
:1058F0000F2071D5B307AF401397570063550722A8
:10590000B307E5410149AE8451B7E30005F0638A6E
:10591000BE0AE35410FD9307F00F6381F608B70742
:1059200000045D8D31B7635E1009630108089307B9
:10593000F00F6385F606B70700045D8DED4763C081
:10594000171F13070002330717413317E500B3573A
:1059500015013337E000D98FFA9713975700635C2E
:10596000070805091307F00F630BE90AB706007E65
:1059700013D71700FD16858B758FD98F01BF33079D
:10598000D84063950610630D0F147D176303071A43
:105990009307F00F6314F810AE84328E630F0E0677
:1059A000814E9306F00FB707400011BF39C9FD18AB
:1059B000B307AF00E38308FA9307F00FE390F6F81C
:1059C000F1BF63990808138916001377E90F63166E
:1059D0000712639B061063030F16E30205EEB3077D
:1059E000AF0013975700014963570700370700FCC2
:1059F0007D17F98F054913F77700E31C07E813DEDD
:105A000037009307F00FE30BF9F893179E00A58377
:105A10009376F90F93FE14005DB593FE1400930680
:105A2000F00F814769BD370700FC7D17F98F13F729
:105A300077003309A940E31E07E4D1B73304AF4030
:105A40009317540063C3070CE31C04E0814E8146A6
:105A50008147B5B53307D840B5C69307F00FE30EBD
:105A6000F8F2B7070004336FFF00ED4763CDE70C92
:105A700093070002998FB317FF003357EF00B33736
:105A8000F0005D8FB307A7004289C1BD9307F00FF7
:105A9000E304F8F0B7070004336FFF00ED4763C27B
:105AA000E70893070002998FB317FF003357EF0001
:105AB000B337F000D98FB307F5404289AE8449BBB4
:105AC000854769B3630E0F067D17B307AF004289A0
:105AD000E30507E89307F00FE319F8F8328E7DBD70
:105AE000328E4289AE8431BFE3090FEAE30805EA4A
:105AF00045BD0DCDAE8EB287D9B39307F00FE3004D
:105B0000F9F2B307AF008583FDB53304E541AE84F8
:105B100081BBE31D0FFCE30505E8AE84BDBD8547F1
:105B200025BD854749BF0149E39707EC814E814771
:105B300079B3B307E5414289AE8419BBB28741B35B
:105B4000328E42897DBD054735BF37068000135729
:105B500075019307F6FF1377F70F9305E007B3F688
:105B6000A7009357F50163FCE5009305D00963FA9C
:105B7000E500370500801345F5FF3E95828001451D
:105B8000828093055009D18E63CDE500130660092C
:105B90003307E64033D7E6003305E040F5F33A85B6
:105BA00082801307A7F63397E600FDB713577501F8
:105BB000370680009307F6FF1377F70F9305E0078A
:105BC000B3F6A7009357F501014563F4E50099C3C7
:105BD000828082809307E0097D55E3EBE7FE930521
:105BE0005009B3E7C60063D7E5001307A7F633955E
:105BF000E7008280130560093307E54033D5E700ED
:105C00008280411106C622C426C20DCD9357F541AC
:105C100033C4A7001D8CAA842285492E9307E0096E
:105C20003387A74093076009FD8063CCE702A14654
:105C30009377F70F63D5A60061153314A4002604EB
:105C4000258021A0814481470144260413559400F6
:105C5000B2402244DE07FE045D8D458D9244410131
:105C600082809307900963DDE7009307B5019546AD
:105C7000B317F400898E3354D400B337F0005D8C31
:105C8000954763D6A7009307B5FF3314F400B70612
:105C900000FCFD16937774003376D40085C39377A8
:105CA000F4009145638CB70011069317560063D733
:105CB00007009307F009758E3387A7401314660019
:105CC00025809377F70F51B7411106C622C415CD31
:105CD0002A84E92C9307E0093387A74093076009DA
:105CE00063C0E704A1469377F70F63D5A60061155B
:105CF0003314A40026042580260413559400B240D2
:105D00002244DE075D8D4101828001442604135543
:105D10009400B24022448147DE075D8D41018280BC
:105D20009307900963DDE7009307B5019546B31724
:105D3000F400898EB337F0003354D4005D8C95475E
:105D400063D6A7009307B5FF3314F400B70600FC31
:105D5000FD16937774003376D40085C39377F400EF
:105D60009145638CB70011069317560063D707005F
:105D70009307F009758E3387A740131466002580BA
:105D8000260413559400B24022449377F70FDE07A0
:105D90005D8D41018280135775011377F70F411113
:105DA0009307170022C426C21314950006C693F762
:105DB000E70F25809354F50185C7935734001307E7
:105DC00007387604B2075207B1831395F401D98FCF
:105DD000C98FB240228522449244BE85410182800F
:105DE00005EB39C42285D922A94763C6A7042D47EC
:105DF000098F930755013357E4003314F4009317C8
:105E0000C70013079038098FB1831377F77F5DBF01
:105E100001CC13573400B7070800D98FB2077604B6
:105E2000B1831307F07F79BF1307F07F814759BF14
:105E30000147814741BF130755FF3317E400014471
:105E40007DBF93D645019397C50093F6F67FB18346
:105E5000138616008E071357D5011376E67FFD8152
:105E60005D8F9318350035CE138806C89307E00F71
:105E700063DD07018147139597009306F00FDE0657
:105E80002581FE05558D4D8D82806355000B93173E
:105E900065000E07B337F000D98F93D8D801B3E768
:105EA000170113F777006301071013F7F700914606
:105EB0006303D7009107370700047D8F75C7130769
:105EC00018001306F00F9376F70FE305C7FA9A0749
:105ED000A58313959700DE062581FE05558D4D8D12
:105EE0008280B367170199EE85CF95479A07A583FE
:105EF0001395970093F6F60FDE062581FE05558D66
:105F00004D8D8280A5DBB70740001395970093065F
:105F1000F00FDE0681452581FE05558D4D8D828071
:105F20008147139597008146DE062581FE05558D34
:105F30004D8D8280A5576348F804F94737068000E5
:105F4000B38707417D45598E6351F504795733076F
:105F50000741130500023357E6006388A7009386C4
:105F600026CAB316D600B3E8D800B3371001D98FCC
:105F700013F77700014815FB139757008546E34850
:105F800007F48146A5B781468DB7938626C8339717
:105F9000D8003337E000B316D600B3D8F800B367A3
:105FA000D700B3E7F800E9B7C28689B7C167637C59
:105FB000F5029307F00F1307000263EBA700972782
:105FC0000000938727C0AA9788233305A7408280C3
:105FD0002181972700009387E7BEAA97882361470E
:105FE0003305A7408280B7070001636DF50061812A
:105FF00097270000938707BDAA9788232147330579
:10600000A74082804181972700009387A7BBAA976A
:10601000882341473305A7408280B3C7A5008D8BF5
:106020003307C50081E78D4763EDC700AA87637E0C
:10603000E508942185078505A38FD7FEE3EBE7FEEE
:10604000828093763500AA8789CA942185078505C1
:10605000A38FD7FE93F63700C5BF9376C7FF13868D
:1060600006FE63F0C70683A3050083A2450083AF45
:10607000850003AFC50083AE050103AE450103A350
:10608000850183A8C5019385450223A0770003A855
:10609000C5FF23A2570023A4F70123A6E70123A8E5
:1060A000D70123AAC70123AC670023AE170193874A
:1060B000470223AE07FF75B790419107910523AEC4
:1060C000C7FEE3EBD7FEE3E6E7F6828039713EDAFE
:1060D0002ED232D436D63AD842DC46DE938781813E
:1060E00022CC804326CA06CEAA8409C41C4C99E35C
:1060F0002285E12B0C4454102686228536C6EF00FB
:10610000D021F2406244D24421618280011126CA2A
:106110004AC806CE22CC4EC652C4AA842E8901C5D6
:106120001C4D91E35D239C4C804499E32685712BA3
:1061300097270000938707BB631BF402C0405E24CF
:10614000A18BB1C71C48A1C7FD59294A1C448345EE
:106150000900FD17B1E91CC463DD07062286A945C5
:1061600026859522FD576308F502294535A0972716
:106170000000938727B96314F4008044C9B79727B8
:106180000000938727B4E31CF4FAC0444DBFA285F6
:106190002685C52A55D97D55F2406244D2444249EC
:1061A000B249224A056182801CC4050963D70700F1
:1061B000184C63CAE700638845011C401387170029
:1061C00018C08CA361B722862685F528E31035F91F
:1061D000D9B71C401387170018C0294798A371B777
:1061E00093878181AA8588436FF05FF2411193877D
:1061F000818122C4804326C206C61C5CAA848DEB22
:1062000061452527B737CDAB08DC9387E7301CC144
:10621000B7176DE6938747235CC1B7E705009387FF
:10622000C7EE1CC5AD475EA50547814718C95CC9C7
:106230001C5CB240224484CB23AA07009244410153
:10624000828041119387818122C4804306C61C5CF1
:106250008DEB6145D92DB737CDAB08DC9387E7309F
:106260001CC1B7176DE6938747235CC1B7E70500EC
:106270009387C7EE1CC5AD475EA50547814718C982
:106280005CC9105C3787954CB7F75158144A484A97
:106290001307D7F29387D742B387F602B24022445E
:1062A0003305E5023E95B387E60233B7E6029386EF
:1062B000170014CA2A9733B5F6003A9548CA06055E
:1062C000058141018280011122CC26CA4AC806CE2E
:1062D0004EC6AA842E89328401C51C4D91E3F52651
:1062E00097270000938707A06317F406C0401C4C53
:1062F0001CC45E24A18BC1C31C48B5CF1C480840F8
:106300009379F90F1379F90F1D8D5C486346F500F9
:10631000A2852685692C25E51C440505FD171CC4AE
:106320001C401387170018C0238037015C4863881E
:10633000A7005E24858B81CBA9476316F900A2854F
:106340002685B5240DEDF24062444A85D244424987
:10635000B24905618280972700009387A79A63144A
:10636000F400804469B7972700009387A795E3104E
:10637000F4F8C044ADBFA2852685212041D17D59C6
:10638000D9B741119387818126C2844322C44AC070
:1063900006C62A892E8489C49C4C99E32685352615
:1063A0009727000093870794631BF402C0400317EC
:1063B000C40093170701C18393F68700ADEA93F6F3
:1063C000070195EEA5472320F900136707045AA497
:1063D0007D55B24022449244024941018280972770
:1063E0000000938727926314F4008044C9B797276D
:1063F00000009387278DE31CF4FAC0444DBF918BB6
:106400009DC34C5889C9930744046384F5004A85A9
:106410001523232A04025E242322040093F7B7FDE8
:106420005EA41C481CC05E2493E787005EA41C4841
:1064300099EB5E241307002093F707286385E70094
:10644000A2854A8591295E2413F717001DC35C4875
:1064500023240400B307F0401CCC1C480145B5FBC5
:106460008317C40013F707082DD793E707045EA42A
:1064700085B7898B014791E3584818C4F9BFDE25D9
:10648000011122CC26CA06CE4AC84EC613F7870091
:10649000AA842E8479EBD841634DE000B841634A69
:1064A000E0000145F2406244D2444249B2490561EC
:1064B000828058547DD703A904009396370123A006
:1064C000040063DB060670485E24918B99C75C402C
:1064D0001D8E5C5899C33C401D8E5C540C50814607
:1064E00026858297FD575A24631DF5009440F54791
:1064F00063E8D706B70740208507B3D7D700858B59
:10650000A5C31C48232204001CC09317370163D87D
:106510000700FD576314F5009C4091E368C84C5890
:1065200023A02401BDDD930744046384F500268580
:106530001121232A0402B5B70C5001468546268551
:106540000297FD572A86E311F5F89C40B5DF7547A1
:106550006385E70059476393E70423A0240191B7BB
:10656000136707045AA47D5535BF83A90501E38A43
:1065700009F203A905008D8B23A0350133093941A8
:10658000014791E3D84918C4E35D20F11C540C5035
:10659000CA864E86268582976347A0005E2493E7CD
:1065A00007045EA4C9B7AA993309A940F1BF9C4961
:1065B000A5C3011122CC06CE2A8411C51C4D81E74A
:1065C0002EC62122B245971700009387A771639CBE
:1065D000F5004C408397C5009DC722856244F24078
:1065E00005616FF0DFE9971700009387A771639447
:1065F000F5000C44C5B7971700009387A76CE39B81
:10660000F5FC4C44C1BFF240624401450561828003
:1066100001458280411122C406C62A844EA572A576
:10662000232005002322050023240500232205063C
:1066300023280500232A0500232C05002146814537
:106640001305C505EF90DFB597170000938727B3B3
:106650005CD097170000938747B51CD497170000AC
:10666000938727B95CD497170000938787BB00D026
:106670001CD8B240224441018280970500009385D6
:1066800045F391AA411126C2130680069384F5FFB3
:10669000B384C4024AC02E8922C406C69385440727
:1066A000352E2A8401CD2320050023222501310522
:1066B00008C4138684068145EF909FAE2285B240C0
:1066C000224492440249410182801C4DA5E74111B8
:1066D00006C622C497070000938767FA1CD59387E4
:1066E000C1819C4323240504232605042328050493
:1066F0006314F50085471CCD2A84352848C02285BF
:106700001D2808C42285052848C4484001469145F3
:10671000EFF05FF008440546A545EFF0BFEF4844B1
:106720000946C945EFF01FEF85471CCCB240224413
:1067300041018280828041119387C18126C28443B6
:106740004AC006C69C4C22C42A8981E72685EFF000
:10675000DFF7938484048044DC40FD1763D6070090
:106760009C40B9CF8440C5BF0317C40039E7C17747
:106770008507232204062320040023220400232467
:1067800004005CC423280400232A0400232C0400F2
:10679000214681451305C405EF909FA0232A0402DA
:1067A000232C040223240404232604042285B2405B
:1067B000224492440249410182801304840671BF3D
:1067C00091454A85EFF01FEC88C049FDB147232071
:1067D000F9000144E1BF797122D44AD052CC56CAA3
:1067E0005AC85EC606D626D24ECE2A8AAE8A130470
:1067F00085040149054BFD5B09ECB25022544A85E2
:1068000092540259F249624AD24A424BB24B456114
:106810008280044483294400FD1963D409000040A8
:10682000E1BFDE24637BFB008397E400638777018D
:10683000A6855285829A3369A90093848406E9BFAC
:106840001971A6DAAE848395E500A2DC86DE328477
:1068500063DB0500DE2423A0060093F7070885E725
:10686000930700401DA0300836C6EF001021B24645
:10687000E34205FE7247BD67F98F7977BA9793B700
:1068800017009CC2F1BF930700041CC0F650665469
:10689000D654014509618280DE25011122CC06CE45
:1068A00026CA4AC8898B2E8489CF930774041CC0DA
:1068B0001CC885475CC8F2406244D2444249056125
:1068C000828074003000AA84EFF09FF7A2452A89E5
:1068D0002685292219E98317C40013F7072061FFD1
:1068E000F19B93E727005EA4C9B797070000938741
:1068F00007D99CD45E2408C008C893E707085EA4A3
:10690000A2475CC8B24781CF8315E4002685EF001B
:10691000701911C55E24F19B93E717005EA45E24F5
:106920003369F9002316240179B793878181AA85F9
:1069300088436DA0DDC183A7C5FF411122C406C6EF
:1069400026C21384C5FF63D307003E94AA84EF00D8
:10695000301C938701899C4381EF2322040023A8E4
:1069600081882244B2402685924441016F00701A0A
:10697000637EF40014403307D4006396E700984325
:10698000DC43369718C05CC0D9BFBA87D84319C357
:10699000E37DE4FE94433386D700631F86001040F6
:1069A000B29694C33386D700E31DC7FA1043584309
:1069B000B29694C3D8C375B76375C400B1479CC081
:1069C0004DB71040B306C4006316D70014435843B4
:1069D000B29614C058C0C0C369B78280011126CADC
:1069E00093843500F19806CE22CC4AC84EC6A10445
:1069F000B14763F3F404B14463E2B4042A89EF00BD
:106A000030119387018998433A8439E0938741890B
:106A10009C4391E781454A85252F23AAA188A68515
:106A20004A853D27FD5963193507B1472320F900F1
:106A30004A85EF00100E29A0E3D004FCB1471CC129
:106A40000145F2406244D2444249B2490561828024
:106A50001C40858F63CF0702AD4663F6F6001CC06D
:106A60003E9404C031A05C406313870223A8F188E0
:106A70004A85EF00100A1305B4009307440061999A
:106A80003307F5405DDF3A94898F1CC05DBF5CC35E
:106A9000C5B72287404095BF130435007198E302C3
:106AA00085FCB305A4404A856525E31C35FBB5BFCD
:106AB0001C46FD171CC663DA0700184E63C5E700C5
:106AC000A9476394F5006FF01F801C422E85138741
:106AD000170018C28CA38280011122CC26CA4AC892
:106AE0004EC652C406CE2A89AE893284B304D6007B
:106AF0007D5A63149400014509A80C204E864A85EE
:106B0000EFF01FFB0504E31645FFF2406244D24458
:106B10004249B249224A05618280357122CD26CB95
:106B20004AC94EC706CF52C556C35AC1DEDEE2DCA3
:106B3000E6DAAA89AE843289368409C51C4D99E308
:106B4000EFF0BFB8971700009387C7196398F40C4C
:106B500083A44900DE24A18BE5C79C48F5C39307B5
:106B60000002A304F1029307000302D22305F102FD
:106B700022C6930B5002971A0000938AAA1A054C5A
:106B8000294B4A841C2099C3639F770DB30C244181
:106B9000638E0C00E6864A86A6854E85EFF0DFF30D
:106BA000FD57630FF51C9256E69636D21C2063897A
:106BB000071CFD571309140002C802CE3ECA02CCBE
:106BC000A309010482D483450900154656852D2763
:106BD00013041900C24751E913F7070109C7130746
:106BE0000002A309E10413F7870009C71307B002E5
:106BF000A309E104834609001307A002638FE60698
:106C0000F2474A848146254618209305140013074D
:106C100007FD6377E60AB5CA3ECE85A89717000040
:106C20009387470E6395F40083A4890025B79717CF
:106C3000000093872709E39FF4F083A4C90019BFDC
:106C4000A6854E85EFF0EFF319D97D55FA406A44D9
:106C5000DA444A49BA492A4A9A4A0A4BF65B665CC0
:106C6000D65C0D618280050431BF33055541331573
:106C7000AC00C98F3EC82289B9B732479306470096
:106C8000184336C6634707023ACE18209307E0023E
:106C9000631DF70418309307A002631BF702B24785
:106CA0000904138747009C433AC663C107023ECAE2
:106CB0002DA83307E04093E727003ACE3EC8F1B74E
:106CC000B387670385462E84BA973DBFFD57C5B786
:106CD000050402CA81468147254618209305140001
:106CE000130707FD6374E606F9F20C200D4617152D
:106CF00000001305A503092511CD97170000938700
:106D0000E7021D8D93070004B397A70042450504D1
:106D10005D8D2AC80C201946171500001305450182
:106D2000130914002304B102C12B35C19797FFFF4B
:106D30009387472D95E74247B2471377071009CF4E
:106D400091073EC69257D2973ED225BDB3876703BF
:106D500085462E84BA9751B79D07E19BA107D5B709
:106D6000780097060000938666D726860C084E8525
:106D700097000000E7000000FD572A8AE314F5FCA5
:106D8000DE2493F70704E39207EC1255C1B57800AF
:106D900097060000938686D426860C084E85012A25
:106DA000E1BF797156CA9C49BA8A984522D426D245
:106DB0004ECE52CC06D64AD05AC85EC6AA892E8478
:106DC000B284368A63D3E700BA879CC00347340491
:106DD00019C385079CC01C4093F7070281C79C40DC
:106DE00089079CC00329040013796900631A09000C
:106DF000130B9401FD5B5C449840998F634CF9043C
:106E00001C408346340493F70702B336D000A5EB49
:106E100013063404D2854E85829AFD576303F50428
:106E20001C4011469840998B544481446397C70095
:106E3000B384E64063D3040081441C44184863547F
:106E4000F700998FBE94014969047D5B639824051E
:106E5000014509A885465A86D2854E85829A631EC9
:106E600075017D55B250225492540259F249624A3A
:106E7000D24A424BB24B456182800509ADBF330710
:106E8000D40013060003A301C704034754049387E7
:106E90001600A2978906A381E7049DBF8546228636
:106EA000D2854E85829AE30E65FB050945B7797157
:106EB00022D426D24AD04ECE06D652CC56CA5AC872
:106EC000B689942D930790063289AA842E8413865E
:106ED0003504638DF60263E2D70693078005638667
:106EE000F61863EDD700638E062093073004638E97
:106EF000F60A930A24042301D404C9A09307300698
:106F00006385F60A93074006E395F6FE1C400843A6
:106F100093F6070893054500C5C61C410CC363D80A
:106F200007001307D002B307F040A301E40497164B
:106F30000000938666E0294765A8930700076382EF
:106F4000F61663E5D7029307E0066389F618930700
:106F5000F006E390F6FA0C401C4313F8050813857D
:106F600047006307080608C39C4385A8930750079A
:106F7000E383F6FE930780076389F61293073007D1
:106F8000E399F6F61C43D04181459386470014C32C
:106F900083AA070056858D2601C53305554148C093
:106FA0005C401CC8A301040461A81C43930A240488
:106FB000938647009C4314C32301F4048547D5B747
:106FC00093F607041C410CC3B9DAC207C18781BF1D
:106FD00093F5050408C3C9D99E231307F0066387F8
:106FE000E60E97160000938626D52947A3010404D0
:106FF0004C400CC463C5050008406D9908C099E376
:10700000B28A89CDB28AB3F5E702FD1AB6958C2112
:107010002380BA00B3D5E70263F0E70CA147631EF3
:10702000F7001C40858B91CB58401C4863C7E70094
:1070300093070003A38FFAFEFD1A3306564110C8CA
:107040004E87CA867000A2852685EFF09FD57D5AAF
:10705000631D450B7D55B250225492540259F2499A
:10706000624AD24A424B45618280A382D504971678
:107070000000938666CC0C40084313F805081C41B9
:107080001105630D080208C313F7150001C793E546
:1070900005020CC04147B9FB0C4093F5F5FD0CC04F
:1070A000B1B79C4193E707029CC193078007A302F5
:1070B000F40497160000938666C975BF13F805049B
:1070C00008C3E30308FCC207C1837DBF9716000015
:1070D000938686C6214719BFAE8735B794411C43B6
:1070E000CC4913F80608138547006306080008C357
:1070F0009C438CC339A008C393F606049C43F5DA7D
:107100008EA323280400B28A25BF14485686CA8558
:1071100026858299E30045F51C40898B8DE7B247AF
:107120004844E35AF5F23E853DB785465686CA8502
:1071300026858299E30065F3050A5C443247998FFE
:10714000E345FAFEE9BF014A930A94017D5BF5B776
:10715000411122C42A842E8523A401B606C6EFA0BD
:107160009FB6FD576317F500938781B69C4391C383
:107170001CC0B240224441018280411122C42E84AD
:107180008395E50006C67922634905007C48AA97E5
:107190007CC8B2402244410182805E247D777D1705
:1071A000F98F5EA4FDB7DE25011122CC26CA4AC89C
:1071B0004EC606CE93F70710AA842E843289B6896C
:1071C00091C78395E5008946014609225E247D77B3
:1071D0007D17F98F5EA48315E4006244F240CE86E9
:1071E0004A86B24942492685D244056125A8411103
:1071F00022C42E848395E50006C6C928FD575A246B
:10720000631AF500FD77FD17F98F5EA4B2402244A2
:10721000410182808567D98F5EA468C8C5BF839508
:10722000E50005A8411122C42A842E85B285368640
:1072300023A401B606C6EFA03FA5FD576317F500CE
:10724000938781B69C4391C31CC0B2402244410144
:107250008280411122C42A842E8523A401B606C649
:10726000C520FD576317F500938781B69C4391C3F2
:107270001CC0B240224441018280411122C42A84B0
:107280002E85B28523A401B606C6C920FD57631713
:10729000F500938781B69C4391C31CC0B240224441
:1072A00041018280411122C42A842E8523A401B683
:1072B00006C65D20FD576317F500938781B69C4392
:1072C00091C31CC0B240224441018280411122C4BA
:1072D0002A842E85B285368623A401B606C6592097
:1072E000FD576317F500938781B69C4391C31CC07B
:1072F000B24022444101828093F5F50F2A9663142F
:10730000C500014582801C21E38EB7FE0505C5BF7F
:1073100082808280411122C42A842E85B2853686DD
:1073200023A401B606C6A920FD576317F50093876D
:1073300081B69C4391C31CC0B2402244410182806B
:107340009307800523A4F1B67D55828093078005BD
:1073500023A4F1B67D5582809307800523A4F1B65E
:10736000014582809307800523A4F1B67D55828074
:107370009307800523A4F1B67D55828053797374F9
:10738000656D436C6B3A25640D0A000043686970B3
:1073900049443A253038780D0A00000043616C6991
:1073A0006272617474696F6E5F56616C203A202559
:1073B000640A00000000003F6666663F0000F0437C
:1073C000CDCCCCCCCCCCEC3F696E2074696D312037
:1073D000697271200000000000F07F45000000008D
:1073E0006666666666660A4000000000000010409F
:1073F000000000000000E03F0000000000003440FA
:1074000000000000CF463640000000C0CCCC164043
:107410007B0E710E670E5C0E510E460E3B0E300E4B
:10742000240E180E0C0E000EF30DE70DDA0DCD0D27
:10743000BF0DB20DA40D960D880D790D6A0D5B0D73
:107440004C0D3D0D2D0D1E0D0D0DFD0CED0CDC0C30
:10745000CB0CBA0CA90C970C850C730C610C4F0C5F
:107460003C0C2A0C170C030CF00BDD0BC90BB50BF5
:10747000A10B8D0B780B640B4F0B3A0B260B100BEB
:10748000FB0AE60AD00ABB0AA50A8F0A790A630A30
:107490004D0A370A200A0A0AF409DD09C709B009AA
:1074A000990983096C0955093E0927091109FA0848
:1074B000E308CC08B5089F08880871085A084408F2
:1074C0002D0817080008EA07D307BD07A70791078B
:1074D0007A0765074F07390723070E07F806E30603
:1074E000CE06B906A4068F067A06660651063D0644
:1074F000290615060106EE05DA05C705B405A1053E
:107500008E057B05690556054405320520050F05E6
:10751000FD04EC04DB04CA04B904A804980488043C
:10752000780468045804490439042A041B040C0430
:10753000FE03EF03E103D303C503B703AA039C03D0
:107540008F038203750368035C035003430337030F
:107550002B03200314030903FD02F202E702DC02FD
:10756000D202C702BD02B302A9029F0295028B029A
:10757000820278026F0266025D0254024C024302EC
:107580003B0232022A0222021A0212020A020302F9
:10759000FB01F401ED01E601DE01D701D101CA01D1
:1075A000C301BD01B601B001AA01A4019E01980169
:1075B00092018C01860181017B01760170016B01D2
:1075C000660161015C01570152014D01480144010E
:1075D0003F013B01360132012D0129012501210125
:1075E0001D011901150111010D010A010601020118
:1075F000FF000000062100001421000020210000EF
:107600002C2100008E21000000401C460000C842D2
:1076100000000040000090410000684100000000B0
:107620009A9999999999B93F9A9999999999A93F4C
:107630009A9999999999D93FB81E85EB51B89E3F6F
:1076400017B75138ACC527370AD7A33C00007A4496
:107650000AD7A33B5B494E464F5D205B25733A2515
:10766000645D20526567697374726174696F6E201E
:1076700073756363657373200D0A0D0A00000000C3
:107680005B4552524F525D205B25733A25645D2065
:107690002052656769737465725F4E756D626572BD
:1076A000206572726F723A2578200D0A0D0A00006B
:1076B0005B4552524F525D205B25733A25645D2035
:1076C0002052656769737465725F53746172745F89
:1076D00041646472657373206572726F72203A2020
:1076E0002578200D0A0D0A00696E2077726974658D
:1076F0002072656769737465722000005B494E46AD
:107700004F5D205B25733A25645D2020534C5F520A
:10771000656164526567697374657242617474650A
:107720007279566F6C74616765200D0A0000000065
:107730005B494E464F5D205B25733A25645D2020F2
:10774000534C5F5265616452656769737465724337
:107750006861726743757272656E74200D0A00006D
:107760005B494E464F5D205B25733A25645D2020C2
:10777000534C5F5265616452656769737465724406
:107780006973636861726743757272656E74200D08
:107790000A0000005B494E464F5D205B25733A2589
:1077A000645D2020534C5F52656164526567697364
:1077B00074657244697363686172674D6F73537463
:1077C000617465200D0A0000000020415B494E46AF
:1077D0004F5D205B25733A25645D2020534C5F523A
:1077E0006561645265676973746572486967685357
:1077F0006964654D6F7354656D70657261747572FF
:1078000065200D0A000000005B494E464F5D205B7D
:1078100025733A25645D2020534C5F5265616452A4
:10782000656769737465724D5050544D6F6465207F
:107830000D0A00005B494E464F5D205B25733A25DB
:10784000645D2020534C5F526561645265676973C3
:10785000746572536F6C61724F70656E43697263C9
:10786000756974566F6C74616765200D0A000000BD
:107870005B494E464F5D205B25733A25645D204D84
:10788000617463685F5374617274666C61672073BE
:10789000756363657373200D0A0D0A005B494E46DC
:1078A0004F5D205B25733A25645D204D61746368EC
:1078B0005F6164647265737320737563636573736A
:1078C000200D0A0D0A0000005B494E464F5D205B0B
:1078D00025733A25645D204D617463685F42726F61
:1078E000616463617374616464726573732073753A
:1078F00063636573730D0A0D0A0000005B494E4611
:107900004F5D205B25733A25645D20526561645F9D
:1079100052656769737465720D0A0D0A00000000F4
:107920005B494E464F5D205B25733A25645D2057C9
:10793000726974655F52656769737465720D0A0DCB
:107940000A0000005B494E464F5D205B25733A25D7
:10795000645D204F74686572206672616D65730D99
:107960000A0D0A005B494E464F5D205B25733A25A0
:10797000645D2042726F6164636173745F5363611D
:107980006E0D0A0D0A0000005B494E464F5D205BFC
:1079900025733A25645D205265676973747261745A
:1079A000696F6E5F726571756573740D0A0D0A00FB
:1079B0005B494E464F5D205B25733A25645D20662A
:1079C000756E636F6465206572726F722025780D25
:1079D0000A0D0A0020647574795F726174696F2002
:1079E0003A2025642F31303030200A0020766F7520
:1079F00074203A2025642F313030200A0000000026
:107A000020496F7574203A2025642F313030200AC8
:107A10000000000020496469736F7574203A2025C6
:107A2000642F313030200A00206D6F7354203A20CB
:107A300025642F3130200A00206D6F7353746174F8
:107A400065203A202564200A0000000020302EC363
:107A5000BBD3D0B9A4D7F73B20312EE4B8C1F7C4CB
:107A6000A3CABD3B20322EBAE3C1F7C4A3CABD3BB3
:107A700020332EBAE3D1B9C4A3CABD3B20342EB8FB
:107A8000A1B3E4C4A3CABD3B20352EC3BBD3D0B53C
:107A9000E7B3D8203A202564200A00000000000047
:107AA0007B14AE47E17A843F766F6C7420696E2058
:107AB0003A2025642F313030200A00003333333F21
:107AC000E8C8FFFFDAC7FFFFDAC7FFFFD8C7FFFF2D
:107AD000E0C7FFFFE0C7FFFFA6C7FFFFD8C7FFFF54
:107AE000E0C7FFFFA6C7FFFFE0C7FFFFD8C7FFFF44
:107AF000D4C8FFFFD4C8FFFFD4C8FFFFA6C7FFFF4D
:107B000024D8FFFF4AD7FFFF1ED8FFFF52D7FFFF41
:107B10001ED8FFFF18D7FFFF1ED8FFFF52D7FFFF69
:107B20004AD7FFFF4AD7FFFF18D7FFFF52D7FFFF03
:107B300058D7FFFF58D7FFFF58D7FFFF18D7FFFFD1
:107B40000AD7FFFF0AD7FFFFDED7FFFFBAD8FFFF34
:107B5000DED7FFFFD8D6FFFFDED7FFFFBAD8FFFF83
:107B60000AD7FFFF0AD7FFFFD8D6FFFFBAD8FFFF1B
:107B700018D7FFFF18D7FFFF18D7FFFFD8D6FFFF92
:107B800032DBFFFF80DAFFFF80DAFFFF7EDAFFFFE4
:107B900084DAFFFF84DAFFFF54DAFFFF7EDAFFFFAB
:107BA00084DAFFFF54DAFFFF84DAFFFF7EDAFFFF9B
:107BB00020DBFFFF20DBFFFF20DBFFFF54DAFFFFAE
:107BC0000001020203030303040404040404040484
:107BD0000505050505050505050505050505050555
:107BE0000606060606060606060606060606060635
:107BF0000606060606060606060606060606060625
:107C00000707070707070707070707070707070704
:107C100007070707070707070707070707070707F4
:107C200007070707070707070707070707070707E4
:107C300007070707070707070707070707070707D4
:107C400008080808080808080808080808080808B4
:107C500008080808080808080808080808080808A4
:107C60000808080808080808080808080808080894
:107C70000808080808080808080808080808080884
:107C80000808080808080808080808080808080874
:107C90000808080808080808080808080808080864
:107CA0000808080808080808080808080808080854
:107CB0000808080808080808080808080808080844
:107CC00000000000000000000000000000000000B4
:107CD00000000000000000000000000000000000A4
:107CE0000000000000000000000000000000000094
:107CF0000000000000000000000000000000000084
:107D00000000000000000000000000000000000073
:107D10000000000000000000000000000000000063
:107D2000232D302B20000000686C4C0065666745F1
:107D30004647000030313233343536373839414226
:107D40004344454600000000303132333435363785
:0C7D500038396162636465660000000061
:107D5C0000000000000000000102030406070809EF
:107D6C0000000000010203040102030406070809D5
:107D7C0000000000000000000000000000E8037894
:107D8C00050A00A406DC05B0040A000A0001000183
:107D9C000014005A0046003200000000534C111130
:107DAC00111111111101000100160000300000002A
:107DBC00182A000010000000A2270000A0000000FC
:107DCC006E270000A10000001E270000D00000005C
:107DDC007A290000D1000000DC280000000100001E
:107DEC00E226000001010000A626000002010000AE
:107DFC006A260000030100002E260000040100008A
:107E0C00F025000005010000CC2500000601000053
:107E1C00A2250000000000000300000080250000E7
:107E2C000000000000000000000000000000000046
:107E3C00000000000400000080250000000000008D
:107E4C000000000000000000000000000000000026
:107E5C00E07C0000007D0000C07C00000000000001
:107E6C000000000000000000000000000000000006
:107E7C0000000000000000000000000000000000F6
:107E8C0000000000000000000000000000000000E6
:107E9C0000000000000000000000000000000000D6
:107EAC0000000000000000000000000000000000C6
:107EBC00006CDC0202040608CC0400203333333F90
:107ECC000101010101000000FC000020FC00002069
:00000001FF
